 HeapFilter

 Timestamp is d3392cd7 (reproducible build file hash)

 Preferred load address is 0000000180000000

 Start         Length     Name                   Class
 0001:00000000 00000050H .text$di                CODE
 0001:00000050 00004aa0H .text$mn                CODE
 0001:00004af0 00000036H .text$mn$00             CODE
 0001:00004b26 00000092H .text$x                 CODE
 0002:00000000 000001d8H .idata$5                DATA
 0002:000001d8 00000038H .00cfg                  DATA
 0002:00000210 00000008H .CRT$XCA                DATA
 0002:00000218 00000020H .CRT$XCU                DATA
 0002:00000238 00000008H .CRT$XCZ                DATA
 0002:00000240 00000008H .CRT$XIA                DATA
 0002:00000248 00000008H .CRT$XIC                DATA
 0002:00000250 00000008H .CRT$XIZ                DATA
 0002:00000258 00000008H .CRT$XLA                DATA
 0002:00000260 00000008H .CRT$XLZ                DATA
 0002:00000268 00000008H .CRT$XPA                DATA
 0002:00000270 00000008H .CRT$XPZ                DATA
 0002:00000278 00000008H .CRT$XTA                DATA
 0002:00000280 00000010H .CRT$XTZ                DATA
 0002:00000288 00000000H .gehcont$y              DATA
 0002:00000288 00000000H .gfids$y                DATA
 0002:00000290 00002770H .rdata                  DATA
 0002:00002a00 00000000H .rdata$CastGuardVftablesA DATA
 0002:00002a00 00000000H .rdata$CastGuardVftablesC DATA
 0002:00002a00 00000028H .rdata$T                DATA
 0002:00002a28 000000bcH .rdata$voltmd           DATA
 0002:00002ae4 00000344H .rdata$zzzdbg           DATA
 0002:00002e28 00000008H .rtc$IAA                DATA
 0002:00002e30 00000008H .rtc$IZZ                DATA
 0002:00002e38 00000008H .rtc$TAA                DATA
 0002:00002e40 00000008H .rtc$TZZ                DATA
 0002:00002e48 00000004H .tls                    DATA
 0002:00002e4c 00000004H .tls$                   DATA
 0002:00002e50 00000008H .tls$ZZZ                DATA
 0002:00002e58 000003c8H .xdata                  DATA
 0002:00003220 00000384H .edata                  DATA
 0002:000035a4 0000008cH .idata$2                DATA
 0002:00003630 00000018H .idata$3                DATA
 0002:00003648 000001d8H .idata$4                DATA
 0002:00003820 0000049aH .idata$6                DATA
 0003:00000000 000000b0H .data                   DATA
 0003:000000b0 0001b288H .bss                    DATA
 0004:00000000 00000444H .pdata                  DATA

  Address         Publics by Value              Rva+Base               Lib:Object

 0000:00000000       __AbsoluteZero             0000000000000000     <absolute>
 0000:00000000       ___safe_se_handler_count   0000000000000000     <absolute>
 0000:00000000       ___safe_se_handler_table   0000000000000000     <absolute>
 0000:00000000       __arm64x_extra_rfe_table   0000000000000000     <absolute>
 0000:00000000       __arm64x_extra_rfe_table_size 0000000000000000     <absolute>
 0000:00000000       __arm64x_native_entrypoint 0000000000000000     <absolute>
 0000:00000000       __arm64x_redirection_metadata 0000000000000000     <absolute>
 0000:00000000       __arm64x_redirection_metadata_count 0000000000000000     <absolute>
 0000:00000000       __dynamic_value_reloc_table 0000000000000000     <absolute>
 0000:00000000       __enclave_config           0000000000000000     <absolute>
 0000:00000000       __guard_check_icall_a64n_fptr 0000000000000000     <absolute>
 0000:00000000       __guard_eh_cont_count      0000000000000000     <absolute>
 0000:00000000       __guard_eh_cont_table      0000000000000000     <absolute>
 0000:00000000       __guard_fids_count         0000000000000000     <absolute>
 0000:00000000       __guard_fids_table         0000000000000000     <absolute>
 0000:00000000       __guard_iat_count          0000000000000000     <absolute>
 0000:00000000       __guard_iat_table          0000000000000000     <absolute>
 0000:00000000       __guard_longjmp_count      0000000000000000     <absolute>
 0000:00000000       __guard_longjmp_table      0000000000000000     <absolute>
 0000:00000000       __hybrid_auxiliary_iat     0000000000000000     <absolute>
 0000:00000000       __hybrid_auxiliary_iat_copy 0000000000000000     <absolute>
 0000:00000000       __hybrid_code_map          0000000000000000     <absolute>
 0000:00000000       __hybrid_code_map_count    0000000000000000     <absolute>
 0000:00000000       __x64_code_ranges_to_entry_points 0000000000000000     <absolute>
 0000:00000000       __x64_code_ranges_to_entry_points_count 0000000000000000     <absolute>
 0000:00000100       __guard_flags              0000000000000100     <absolute>
 0000:00000000       __ImageBase                0000000180000000     <linker-defined>
 0001:00000050       ?NewObject@JNIEnv_@@QEAAPEAV_jobject@@PEAV_jclass@@PEAU_jmethodID@@ZZ 0000000180001050 f i libHeapFilter.obj
 0001:00000078       ?SetEventNotificationMode@_jvmtiEnv@@QEAA?AW4jvmtiError@@W4jvmtiEventMode@@W4jvmtiEvent@@PEAV_jobject@@ZZ 0000000180001078 f i libHeapFilter.obj
 0001:00000084       ?TranslateError@@YAPEBDW4jvmtiError@@@Z 0000000180001084 f   libHeapFilter.obj
 0001:0000033c       ?nsk_jni_check_exception@@YAHPEAUJNIEnv_@@QEBDH@Z 000000018000133c f   libHeapFilter.obj
 0001:00000480       ?nsk_jni_lverify@@YAHHPEAUJNIEnv_@@HQEBDH1ZZ 0000000180001480 f   libHeapFilter.obj
 0001:00000520       Agent_Initialize           0000000180001520 f   libHeapFilter.obj
 0001:0000080c       Agent_OnAttach             000000018000180c f   libHeapFilter.obj
 0001:0000080c       Agent_OnLoad               000000018000180c f   libHeapFilter.obj
 0001:00000814       Java_nsk_jvmti_unit_FollowReferences_FollowRefObjects_addRefToVerify 0000000180001814 f   libHeapFilter.obj
 0001:000009ec       Java_nsk_jvmti_unit_FollowReferences_FollowRefObjects_getTag 00000001800019ec f   libHeapFilter.obj
 0001:00000aac       Java_nsk_jvmti_unit_FollowReferences_FollowRefObjects_resetRefsToVerify 0000000180001aac f   libHeapFilter.obj
 0001:00000ab4       Java_nsk_jvmti_unit_FollowReferences_FollowRefObjects_resetTags 0000000180001ab4 f   libHeapFilter.obj
 0001:00000af8       Java_nsk_jvmti_unit_FollowReferences_FollowRefObjects_setTag 0000000180001af8 f   libHeapFilter.obj
 0001:00000d50       Java_nsk_share_jvmti_ArgumentHandler_getAgentOptionsString 0000000180001d50 f   libHeapFilter.obj
 0001:00000e00       Java_nsk_share_jvmti_DebugeeClass_checkStatus 0000000180001e00 f   libHeapFilter.obj
 0001:00000e88       Java_nsk_share_jvmti_DebugeeClass_resetAgentData 0000000180001e88 f   libHeapFilter.obj
 0001:00000ee8       Java_nsk_share_jvmti_RedefineAgent_agentStatus 0000000180001ee8 f   libHeapFilter.obj
 0001:00000ef4       Java_nsk_share_jvmti_RedefineAgent_isRedefined 0000000180001ef4 f   libHeapFilter.obj
 0001:00000f00       Java_nsk_share_jvmti_RedefineAgent_redefineAttempted 0000000180001f00 f   libHeapFilter.obj
 0001:00000f0c       MA_checkStatus             0000000180001f0c f   libHeapFilter.obj
 0001:00000fb0       __local_stdio_printf_options 0000000180001fb0 f i libHeapFilter.obj
 0001:000015f0       array_callback             00000001800025f0 f   libHeapFilter.obj
 0001:000018d4       exitOnError                00000001800028d4 f   libHeapFilter.obj
 0001:00001958       field_callback             0000000180002958 f   libHeapFilter.obj
 0001:00001a68       fprintf                    0000000180002a68 f i libHeapFilter.obj
 0001:00001aac       heap_callback              0000000180002aac f   libHeapFilter.obj
 0001:00001b78       is_primitive_type          0000000180002b78 f   libHeapFilter.obj
 0001:00001c28       nsk_complain               0000000180002c28 f   libHeapFilter.obj
 0001:00001c54       nsk_jvmti_createJVMTIEnv   0000000180002c54 f   libHeapFilter.obj
 0001:00001d84       nsk_jvmti_enableEvents     0000000180002d84 f   libHeapFilter.obj
 0001:00001e58       nsk_jvmti_findOptionValue  0000000180002e58 f   libHeapFilter.obj
 0001:00001ed0       nsk_jvmti_lverify          0000000180002ed0 f   libHeapFilter.obj
 0001:00001fc0       nsk_jvmti_parseOptions     0000000180002fc0 f   libHeapFilter.obj
 0001:00002210       nsk_jvmti_resetAgentData   0000000180003210 f   libHeapFilter.obj
 0001:00002290       nsk_jvmti_resumeSync       0000000180003290 f   libHeapFilter.obj
 0001:00002338       nsk_jvmti_setFailStatus    0000000180003338 f   libHeapFilter.obj
 0001:00002374       nsk_jvmti_waitForSync      0000000180003374 f   libHeapFilter.obj
 0001:00002478       nsk_lcomplain              0000000180003478 f   libHeapFilter.obj
 0001:00002498       nsk_ldisplay               0000000180003498 f   libHeapFilter.obj
 0001:000024b8       nsk_ltrace                 00000001800034b8 f   libHeapFilter.obj
 0001:000024d8       nsk_lvcomplain             00000001800034d8 f   libHeapFilter.obj
 0001:00002690       nsk_lvdisplay              0000000180003690 f   libHeapFilter.obj
 0001:000026dc       nsk_lverify                00000001800036dc f   libHeapFilter.obj
 0001:00002738       nsk_lvtrace                0000000180003738 f   libHeapFilter.obj
 0001:00002798       nsk_printf                 0000000180003798 f   libHeapFilter.obj
 0001:000027c0       nsk_vprintf                00000001800037c0 f   libHeapFilter.obj
 0001:00002874       object_free_callback       0000000180003874 f   libHeapFilter.obj
 0001:000028d4       occurance_expected         00000001800038d4 f   libHeapFilter.obj
 0001:00002924       printf                     0000000180003924 f i libHeapFilter.obj
 0001:00002974       release_object_info        0000000180003974 f   libHeapFilter.obj
 0001:00002a1c       set_expected_value         0000000180003a1c f   libHeapFilter.obj
 0001:00002e2c       string_callback            0000000180003e2c f   libHeapFilter.obj
 0001:000030ec       tag_objects                00000001800040ec f   libHeapFilter.obj
 0001:00003ad4       verify_objects             0000000180004ad4 f   libHeapFilter.obj
 0001:00003b94       verify_tag                 0000000180004b94 f   libHeapFilter.obj
 0001:00003bcc       __raise_securityfailure    0000000180004bcc f   MSVCRT:gs_report.obj
 0001:00003c00       __report_gsfailure         0000000180004c00 f   MSVCRT:gs_report.obj
 0001:00003e40       __GSHandlerCheck           0000000180004e40 f   MSVCRT:gshandler.obj
 0001:00003e60       __GSHandlerCheckCommon     0000000180004e60 f   MSVCRT:gshandler.obj
 0001:00003ed0       __security_check_cookie    0000000180004ed0 f   MSVCRT:amdsecgs.obj
 0001:00004210       _DllMainCRTStartup         0000000180005210 f   MSVCRT:dll_dllmain.obj
 0001:00004250       __scrt_acquire_startup_lock 0000000180005250 f   MSVCRT:utility.obj
 0001:0000428c       __scrt_dllmain_after_initialize_c 000000018000528c f   MSVCRT:utility.obj
 0001:000042c0       __scrt_dllmain_before_initialize_c 00000001800052c0 f   MSVCRT:utility.obj
 0001:000042d8       __scrt_dllmain_crt_thread_attach 00000001800052d8 f   MSVCRT:utility.obj
 0001:00004300       __scrt_dllmain_crt_thread_detach 0000000180005300 f   MSVCRT:utility.obj
 0001:00004318       __scrt_dllmain_exception_filter 0000000180005318 f   MSVCRT:utility.obj
 0001:00004378       __scrt_dllmain_uninitialize_c 0000000180005378 f   MSVCRT:utility.obj
 0001:000043a8       __scrt_dllmain_uninitialize_critical 00000001800053a8 f   MSVCRT:utility.obj
 0001:000043bc       __scrt_initialize_crt      00000001800053bc f   MSVCRT:utility.obj
 0001:00004408       __scrt_initialize_onexit_tables 0000000180005408 f   MSVCRT:utility.obj
 0001:00004494       __scrt_is_nonwritable_in_current_image 0000000180005494 f   MSVCRT:utility.obj
 0001:0000452c       __scrt_release_startup_lock 000000018000552c f   MSVCRT:utility.obj
 0001:00004550       __scrt_uninitialize_crt    0000000180005550 f   MSVCRT:utility.obj
 0001:0000457c       _onexit                    000000018000557c f   MSVCRT:utility.obj
 0001:000045b8       atexit                     00000001800055b8 f   MSVCRT:utility.obj
 0001:000045d0       __crt_debugger_hook        00000001800055d0 f   MSVCRT:utility_desktop.obj
 0001:000045d8       __scrt_fastfail            00000001800055d8 f   MSVCRT:utility_desktop.obj
 0001:00004724       _guard_check_icall_nop     0000000180005724 f i MSVCRT:guard_support.obj
 0001:00004728       __security_init_cookie     0000000180005728 f   MSVCRT:gs_support.obj
 0001:000047d4       DllMain                    00000001800057d4 f   MSVCRT:dll_dllmain_stub.obj
 0001:000047f8       ?__scrt_initialize_type_info@@YAXXZ 00000001800057f8 f   MSVCRT:tncleanup.obj
 0001:00004808       ?__scrt_uninitialize_type_info@@YAXXZ 0000000180005808 f   MSVCRT:tncleanup.obj
 0001:00004814       __local_stdio_scanf_options 0000000180005814 f i MSVCRT:default_local_stdio_options.obj
 0001:0000481c       __scrt_initialize_default_local_stdio_options 000000018000581c f   MSVCRT:default_local_stdio_options.obj
 0001:00004838       __scrt_get_dyn_tls_init_callback 0000000180005838 f   MSVCRT:dyn_tls_init.obj
 0001:00004840       _RTC_Initialize            0000000180005840 f   MSVCRT:initsect.obj
 0001:0000487c       _RTC_Terminate             000000018000587c f   MSVCRT:initsect.obj
 0001:000048b8       __isa_available_init       00000001800058b8 f   MSVCRT:cpu_disp.obj
 0001:00004a64       _get_startup_argv_mode     0000000180005a64 f   MSVCRT:argv_mode.obj
 0001:00004a6c       __scrt_is_ucrt_dll_in_use  0000000180005a6c f   MSVCRT:ucrt_detection.obj
 0001:00004a80       memcpy                     0000000180005a80 f   vcruntime:VCRUNTIME140.dll
 0001:00004a86       memset                     0000000180005a86 f   vcruntime:VCRUNTIME140.dll
 0001:00004a8c       strchr                     0000000180005a8c f   vcruntime:VCRUNTIME140.dll
 0001:00004a92       __C_specific_handler       0000000180005a92 f   vcruntime:VCRUNTIME140.dll
 0001:00004a98       __std_type_info_destroy_list 0000000180005a98 f   vcruntime:VCRUNTIME140.dll
 0001:00004a9e       strcmp                     0000000180005a9e f   ucrt:api-ms-win-crt-string-l1-1-0.dll
 0001:00004aa4       strlen                     0000000180005aa4 f   ucrt:api-ms-win-crt-string-l1-1-0.dll
 0001:00004aaa       _initterm                  0000000180005aaa f   ucrt:api-ms-win-crt-runtime-l1-1-0.dll
 0001:00004ab0       _initterm_e                0000000180005ab0 f   ucrt:api-ms-win-crt-runtime-l1-1-0.dll
 0001:00004ab6       _seh_filter_dll            0000000180005ab6 f   ucrt:api-ms-win-crt-runtime-l1-1-0.dll
 0001:00004abc       _configure_narrow_argv     0000000180005abc f   ucrt:api-ms-win-crt-runtime-l1-1-0.dll
 0001:00004ac2       _initialize_narrow_environment 0000000180005ac2 f   ucrt:api-ms-win-crt-runtime-l1-1-0.dll
 0001:00004ac8       _initialize_onexit_table   0000000180005ac8 f   ucrt:api-ms-win-crt-runtime-l1-1-0.dll
 0001:00004ace       _register_onexit_function  0000000180005ace f   ucrt:api-ms-win-crt-runtime-l1-1-0.dll
 0001:00004ad4       _execute_onexit_table      0000000180005ad4 f   ucrt:api-ms-win-crt-runtime-l1-1-0.dll
 0001:00004ada       _crt_atexit                0000000180005ada f   ucrt:api-ms-win-crt-runtime-l1-1-0.dll
 0001:00004ae0       _cexit                     0000000180005ae0 f   ucrt:api-ms-win-crt-runtime-l1-1-0.dll
 0001:00004ae8       __acrt_initialize          0000000180005ae8 f   MSVCRT:ucrt_stubs.obj
 0001:00004ae8       __acrt_thread_attach       0000000180005ae8 f   MSVCRT:ucrt_stubs.obj
 0001:00004ae8       __acrt_thread_detach       0000000180005ae8 f   MSVCRT:ucrt_stubs.obj
 0001:00004ae8       __acrt_uninitialize        0000000180005ae8 f   MSVCRT:ucrt_stubs.obj
 0001:00004ae8       __acrt_uninitialize_critical 0000000180005ae8 f   MSVCRT:ucrt_stubs.obj
 0001:00004ae8       __scrt_stub_for_acrt_initialize 0000000180005ae8 f   MSVCRT:ucrt_stubs.obj
 0001:00004ae8       __scrt_stub_for_acrt_thread_attach 0000000180005ae8 f   MSVCRT:ucrt_stubs.obj
 0001:00004ae8       __scrt_stub_for_acrt_thread_detach 0000000180005ae8 f   MSVCRT:ucrt_stubs.obj
 0001:00004ae8       __scrt_stub_for_acrt_uninitialize 0000000180005ae8 f   MSVCRT:ucrt_stubs.obj
 0001:00004ae8       __scrt_stub_for_acrt_uninitialize_critical 0000000180005ae8 f   MSVCRT:ucrt_stubs.obj
 0001:00004ae8       __vcrt_initialize          0000000180005ae8 f   MSVCRT:ucrt_stubs.obj
 0001:00004ae8       __vcrt_thread_attach       0000000180005ae8 f   MSVCRT:ucrt_stubs.obj
 0001:00004ae8       __vcrt_thread_detach       0000000180005ae8 f   MSVCRT:ucrt_stubs.obj
 0001:00004ae8       __vcrt_uninitialize        0000000180005ae8 f   MSVCRT:ucrt_stubs.obj
 0001:00004ae8       __vcrt_uninitialize_critical 0000000180005ae8 f   MSVCRT:ucrt_stubs.obj
 0001:00004aec       __scrt_stub_for_is_c_termination_complete 0000000180005aec f   MSVCRT:ucrt_stubs.obj
 0001:00004aec       _is_c_termination_complete 0000000180005aec f   MSVCRT:ucrt_stubs.obj
 0001:00004b00       _guard_dispatch_icall_nop  0000000180005b00 f   MSVCRT:guard_dispatch.obj
 0001:00004b20       _guard_xfg_dispatch_icall_nop 0000000180005b20 f   MSVCRT:guard_xfg_dispatch.obj
 0002:00000000       __imp_RtlCaptureContext    0000000180006000     kernel32:KERNEL32.dll
 0002:00000008       __imp_RtlLookupFunctionEntry 0000000180006008     kernel32:KERNEL32.dll
 0002:00000010       __imp_RtlVirtualUnwind     0000000180006010     kernel32:KERNEL32.dll
 0002:00000018       __imp_UnhandledExceptionFilter 0000000180006018     kernel32:KERNEL32.dll
 0002:00000020       __imp_SetUnhandledExceptionFilter 0000000180006020     kernel32:KERNEL32.dll
 0002:00000028       __imp_GetCurrentProcess    0000000180006028     kernel32:KERNEL32.dll
 0002:00000030       __imp_TerminateProcess     0000000180006030     kernel32:KERNEL32.dll
 0002:00000038       __imp_IsProcessorFeaturePresent 0000000180006038     kernel32:KERNEL32.dll
 0002:00000040       __imp_CloseHandle          0000000180006040     kernel32:KERNEL32.dll
 0002:00000048       __imp_InitializeCriticalSectionAndSpinCount 0000000180006048     kernel32:KERNEL32.dll
 0002:00000050       __imp_DeleteCriticalSection 0000000180006050     kernel32:KERNEL32.dll
 0002:00000058       __imp_CreateEventW         0000000180006058     kernel32:KERNEL32.dll
 0002:00000060       __imp_GetModuleHandleW     0000000180006060     kernel32:KERNEL32.dll
 0002:00000068       __imp_GetProcAddress       0000000180006068     kernel32:KERNEL32.dll
 0002:00000070       __imp_IsDebuggerPresent    0000000180006070     kernel32:KERNEL32.dll
 0002:00000078       __imp_QueryPerformanceCounter 0000000180006078     kernel32:KERNEL32.dll
 0002:00000080       __imp_GetCurrentProcessId  0000000180006080     kernel32:KERNEL32.dll
 0002:00000088       __imp_GetCurrentThreadId   0000000180006088     kernel32:KERNEL32.dll
 0002:00000090       __imp_GetSystemTimeAsFileTime 0000000180006090     kernel32:KERNEL32.dll
 0002:00000098       __imp_DisableThreadLibraryCalls 0000000180006098     kernel32:KERNEL32.dll
 0002:000000a0       __imp_InitializeSListHead  00000001800060a0     kernel32:KERNEL32.dll
 0002:000000a8       \177KERNEL32_NULL_THUNK_DATA 00000001800060a8     kernel32:KERNEL32.dll
 0002:000000b0       __imp_memcpy               00000001800060b0     vcruntime:VCRUNTIME140.dll
 0002:000000b8       __imp_memset               00000001800060b8     vcruntime:VCRUNTIME140.dll
 0002:000000c0       __imp_strchr               00000001800060c0     vcruntime:VCRUNTIME140.dll
 0002:000000c8       __imp___C_specific_handler 00000001800060c8     vcruntime:VCRUNTIME140.dll
 0002:000000d0       __imp___std_type_info_destroy_list 00000001800060d0     vcruntime:VCRUNTIME140.dll
 0002:000000d8       \177VCRUNTIME140_NULL_THUNK_DATA 00000001800060d8     vcruntime:VCRUNTIME140.dll
 0002:000000e0       __imp_strtol               00000001800060e0     ucrt:api-ms-win-crt-convert-l1-1-0.dll
 0002:000000e8       \177api-ms-win-crt-convert-l1-1-0_NULL_THUNK_DATA 00000001800060e8     ucrt:api-ms-win-crt-convert-l1-1-0.dll
 0002:000000f0       __imp_malloc               00000001800060f0     ucrt:api-ms-win-crt-heap-l1-1-0.dll
 0002:000000f8       __imp_free                 00000001800060f8     ucrt:api-ms-win-crt-heap-l1-1-0.dll
 0002:00000100       __imp_calloc               0000000180006100     ucrt:api-ms-win-crt-heap-l1-1-0.dll
 0002:00000108       \177api-ms-win-crt-heap-l1-1-0_NULL_THUNK_DATA 0000000180006108     ucrt:api-ms-win-crt-heap-l1-1-0.dll
 0002:00000110       __imp__errno               0000000180006110     ucrt:api-ms-win-crt-runtime-l1-1-0.dll
 0002:00000118       __imp_exit                 0000000180006118     ucrt:api-ms-win-crt-runtime-l1-1-0.dll
 0002:00000120       __imp__cexit               0000000180006120     ucrt:api-ms-win-crt-runtime-l1-1-0.dll
 0002:00000128       __imp__crt_atexit          0000000180006128     ucrt:api-ms-win-crt-runtime-l1-1-0.dll
 0002:00000130       __imp__execute_onexit_table 0000000180006130     ucrt:api-ms-win-crt-runtime-l1-1-0.dll
 0002:00000138       __imp__register_onexit_function 0000000180006138     ucrt:api-ms-win-crt-runtime-l1-1-0.dll
 0002:00000140       __imp__initialize_onexit_table 0000000180006140     ucrt:api-ms-win-crt-runtime-l1-1-0.dll
 0002:00000148       __imp__initialize_narrow_environment 0000000180006148     ucrt:api-ms-win-crt-runtime-l1-1-0.dll
 0002:00000150       __imp__configure_narrow_argv 0000000180006150     ucrt:api-ms-win-crt-runtime-l1-1-0.dll
 0002:00000158       __imp__seh_filter_dll      0000000180006158     ucrt:api-ms-win-crt-runtime-l1-1-0.dll
 0002:00000160       __imp__initterm_e          0000000180006160     ucrt:api-ms-win-crt-runtime-l1-1-0.dll
 0002:00000168       __imp__initterm            0000000180006168     ucrt:api-ms-win-crt-runtime-l1-1-0.dll
 0002:00000170       \177api-ms-win-crt-runtime-l1-1-0_NULL_THUNK_DATA 0000000180006170     ucrt:api-ms-win-crt-runtime-l1-1-0.dll
 0002:00000178       __imp___acrt_iob_func      0000000180006178     ucrt:api-ms-win-crt-stdio-l1-1-0.dll
 0002:00000180       __imp_fflush               0000000180006180     ucrt:api-ms-win-crt-stdio-l1-1-0.dll
 0002:00000188       __imp___stdio_common_vsprintf 0000000180006188     ucrt:api-ms-win-crt-stdio-l1-1-0.dll
 0002:00000190       __imp___stdio_common_vfprintf 0000000180006190     ucrt:api-ms-win-crt-stdio-l1-1-0.dll
 0002:00000198       \177api-ms-win-crt-stdio-l1-1-0_NULL_THUNK_DATA 0000000180006198     ucrt:api-ms-win-crt-stdio-l1-1-0.dll
 0002:000001a0       __imp_wcslen               00000001800061a0     ucrt:api-ms-win-crt-string-l1-1-0.dll
 0002:000001a8       __imp_strcmp               00000001800061a8     ucrt:api-ms-win-crt-string-l1-1-0.dll
 0002:000001b0       __imp__strdup              00000001800061b0     ucrt:api-ms-win-crt-string-l1-1-0.dll
 0002:000001b0       __imp_strdup               00000001800061b0     ucrt:api-ms-win-crt-string-l1-1-0.dll
 0002:000001b8       __imp_strlen               00000001800061b8     ucrt:api-ms-win-crt-string-l1-1-0.dll
 0002:000001c0       __imp_strpbrk              00000001800061c0     ucrt:api-ms-win-crt-string-l1-1-0.dll
 0002:000001c8       __imp_strncpy              00000001800061c8     ucrt:api-ms-win-crt-string-l1-1-0.dll
 0002:000001d0       \177api-ms-win-crt-string-l1-1-0_NULL_THUNK_DATA 00000001800061d0     ucrt:api-ms-win-crt-string-l1-1-0.dll
 0002:000001d8       __guard_check_icall_fptr   00000001800061d8     MSVCRT:guard_support.obj
 0002:000001e0       __guard_xfg_check_icall_fptr 00000001800061e0     MSVCRT:guard_support.obj
 0002:000001e8       __guard_dispatch_icall_fptr 00000001800061e8     MSVCRT:guard_support.obj
 0002:000001f0       __guard_xfg_dispatch_icall_fptr 00000001800061f0     MSVCRT:guard_support.obj
 0002:000001f8       __guard_xfg_table_dispatch_icall_fptr 00000001800061f8     MSVCRT:guard_support.obj
 0002:00000200       __castguard_check_failure_os_handled_fptr 0000000180006200     MSVCRT:guard_support.obj
 0002:00000208       __guard_memcpy_fptr        0000000180006208     vcruntime:softmemtag.obj
 0002:00000210       __xc_a                     0000000180006210     MSVCRT:initializers.obj
 0002:00000238       __xc_z                     0000000180006238     MSVCRT:initializers.obj
 0002:00000240       __xi_a                     0000000180006240     MSVCRT:initializers.obj
 0002:00000250       __xi_z                     0000000180006250     MSVCRT:initializers.obj
 0002:00000258       __xl_a                     0000000180006258     MSVCRT:tlssup.obj
 0002:00000260       __xl_z                     0000000180006260     MSVCRT:tlssup.obj
 0002:00000268       __xp_a                     0000000180006268     MSVCRT:initializers.obj
 0002:00000270       __xp_z                     0000000180006270     MSVCRT:initializers.obj
 0002:00000278       __xt_a                     0000000180006278     MSVCRT:initializers.obj
 0002:00000280       __xt_z                     0000000180006280     MSVCRT:initializers.obj
 0002:00000290       g_refKindStr               0000000180006290     libHeapFilter.obj
 0002:00000440       ??_C@_09BPLDFGCI@unknown_0@ 0000000180006440     libHeapFilter.obj
 0002:00000450       ??_C@_0BL@FPNMECJD@JVMTI_HEAP_REFERENCE_CLASS@ 0000000180006450     libHeapFilter.obj
 0002:00000470       ??_C@_0BL@FKGKKLNM@JVMTI_HEAP_REFERENCE_FIELD@ 0000000180006470     libHeapFilter.obj
 0002:00000490       ??_C@_0CD@CAEHCFJF@JVMTI_HEAP_REFERENCE_ARRAY_ELEM@ 0000000180006490     libHeapFilter.obj
 0002:000004b8       ??_C@_0CC@DNEBMCNK@JVMTI_HEAP_REFERENCE_CLASS_LOAD@ 00000001800064b8     libHeapFilter.obj
 0002:000004e0       ??_C@_0BN@CJMIPEBB@JVMTI_HEAP_REFERENCE_SIGNERS@ 00000001800064e0     libHeapFilter.obj
 0002:00000500       ??_C@_0CH@HBOIDPEB@JVMTI_HEAP_REFERENCE_PROTECTION@ 0000000180006500     libHeapFilter.obj
 0002:00000528       ??_C@_0BP@MDKGDGKL@JVMTI_HEAP_REFERENCE_INTERFACE@ 0000000180006528     libHeapFilter.obj
 0002:00000548       ??_C@_0CC@JJMIHNJH@JVMTI_HEAP_REFERENCE_STATIC_FIE@ 0000000180006548     libHeapFilter.obj
 0002:00000570       ??_C@_0CD@IDHEEGID@JVMTI_HEAP_REFERENCE_CONSTANT_P@ 0000000180006570     libHeapFilter.obj
 0002:00000598       ??_C@_0CA@EFFCHNG@JVMTI_HEAP_REFERENCE_SUPERCLASS@ 0000000180006598     libHeapFilter.obj
 0002:000005b8       ??_C@_0L@PCDFHGCJ@unknown_11@ 00000001800065b8     libHeapFilter.obj
 0002:000005c8       ??_C@_0L@NJBICFOK@unknown_12@ 00000001800065c8     libHeapFilter.obj
 0002:000005d8       ??_C@_0L@MAADBEKL@unknown_13@ 00000001800065d8     libHeapFilter.obj
 0002:000005e8       ??_C@_0L@IPECICGM@unknown_14@ 00000001800065e8     libHeapFilter.obj
 0002:000005f8       ??_C@_0L@JGFJLDCN@unknown_15@ 00000001800065f8     libHeapFilter.obj
 0002:00000608       ??_C@_0L@LNHEOAOO@unknown_16@ 0000000180006608     libHeapFilter.obj
 0002:00000618       ??_C@_0L@KEGPNBKP@unknown_17@ 0000000180006618     libHeapFilter.obj
 0002:00000628       ??_C@_0L@CDPHMNGA@unknown_18@ 0000000180006628     libHeapFilter.obj
 0002:00000638       ??_C@_0L@DKOMPMCB@unknown_19@ 0000000180006638     libHeapFilter.obj
 0002:00000648       ??_C@_0L@OJGIPJDB@unknown_20@ 0000000180006648     libHeapFilter.obj
 0002:00000658       ??_C@_0CA@KAOFNDEM@JVMTI_HEAP_REFERENCE_JNI_GLOBAL@ 0000000180006658     libHeapFilter.obj
 0002:00000678       ??_C@_0CC@HPFAJBK@JVMTI_HEAP_REFERENCE_SYSTEM_CLA@ 0000000180006678     libHeapFilter.obj
 0002:000006a0       ??_C@_0BN@FDEGFOHC@JVMTI_HEAP_REFERENCE_MONITOR@ 00000001800066a0     libHeapFilter.obj
 0002:000006c0       ??_C@_0CB@HKIBCMAJ@JVMTI_HEAP_REFERENCE_STACK_LOCA@ 00000001800066c0     libHeapFilter.obj
 0002:000006e8       ??_C@_0BP@EAACMMOE@JVMTI_HEAP_REFERENCE_JNI_LOCAL@ 00000001800066e8     libHeapFilter.obj
 0002:00000708       ??_C@_0BM@IJDEOGOE@JVMTI_HEAP_REFERENCE_THREAD@ 0000000180006708     libHeapFilter.obj
 0002:00000728       ??_C@_0BL@EDGPPKC@JVMTI_HEAP_REFERENCE_OTHER@ 0000000180006728     libHeapFilter.obj
 0002:00000744       ??_C@_04BCJPDBDA@Code@     0000000180006744     libHeapFilter.obj
 0002:00000750       ??_C@_0BA@OCLMCFKC@LineNumberTable@ 0000000180006750     libHeapFilter.obj
 0002:00000760       ??_C@_0BD@CPAEPILC@LocalVariableTable@ 0000000180006760     libHeapFilter.obj
 0002:00000778       ??_C@_0BH@NMBDNHBD@LocalVariableTypeTable@ 0000000180006778     libHeapFilter.obj
 0002:00000790       ??_C@_0O@HIHEEDNJ@StackMapTable@ 0000000180006790     libHeapFilter.obj
 0002:000007a0       ??_C@_1CI@CAPMLGKG@?$AAI?$AA?8?$AAm?$AA?5?$AAa?$AA?5?$AAt?$AAa?$AAg?$AAg?$AAe?$AAd?$AA?5?$AAs?$AAt@ 00000001800067a0     libHeapFilter.obj
 0002:000007c8       ??_C@_1CO@GOLPFBAK@?$AAI?$AA?8?$AAm?$AA?5?$AAa?$AAn?$AA?5?$AAu?$AAn?$AAt?$AAa?$AAg?$AAg?$AAe?$AAd@ 00000001800067c8     libHeapFilter.obj
 0002:000007f8       ??_C@_0L@HCDIAMJG@?9?5?$CFs?0?5?$CFd?3?5@ 00000001800067f8     libHeapFilter.obj
 0002:00000810       ??_C@_0JI@HLPECLFI@?$CD?5?4?4?4?6?$CD?5ERROR?3?5too?5many?5complai@ 0000000180006810     libHeapFilter.obj
 0002:000008b0       ??_C@_0ED@JNEKCCOB@The?5following?5fake?5exception?5st@ 00000001800068b0     libHeapFilter.obj
 0002:000008f8       ??_C@_0CN@FCNMDFBH@nsk?4share?4Fake_Exception_for_RU@ 00000001800068f8     libHeapFilter.obj
 0002:00000928       ??_C@_08PGFFNAEI@?$CI?$CFs?3?$CFd?$CJ?5@ 0000000180006928     libHeapFilter.obj
 0002:00000938       ??_C@_0DP@IENMAEGI@s?2test?2hotspot?2jtreg?2vmTestbase@ 0000000180006938     libHeapFilter.obj
 0002:00000978       ??_C@_0BL@NDJLFFJB@?7at?5nsk_lvcomplain?$CI?$CFs?3?$CFd?$CJ?6@ 0000000180006978     libHeapFilter.obj
 0002:00000998       ??_C@_0BC@JOOKAFKF@?$CD?5ERROR?3?5?$CFs?0?5?$CFd?3?5@ 0000000180006998     libHeapFilter.obj
 0002:000009b0       ??_C@_09KJEAHMEH@?$CD?5ERROR?3?5@ 00000001800069b0     libHeapFilter.obj
 0002:000009bc       ??_C@_02GPIOPFAK@?$DO?$DO@ 00000001800069bc     libHeapFilter.obj
 0002:000009c0       ??_C@_02FODMEDOG@?$DM?$DM@ 00000001800069c0     libHeapFilter.obj
 0002:000009c4       ??_C@_02DJGKEECL@?4?4@     00000001800069c4     libHeapFilter.obj
 0002:000009c8       ??_C@_0O@CJPGJOAF@?9?5?$CFs?0?5?$CFd?3?5?$CFs?5@ 00000001800069c8     libHeapFilter.obj
 0002:000009d8       ??_C@_0CB@IAKPDOIC@?$CD?5?5?5verified?5assertion?5is?5FALSE@ 00000001800069d8     libHeapFilter.obj
 0002:00000a00       ??_C@_0CO@LGONDEPD@stdout?3?5fflush?5failed?5?9?5err?$DN?$CFd?5@ 0000000180006a00     libHeapFilter.obj
 0002:00000a30       ??_C@_0CO@KBGKJPBD@stderr?3?5fflush?5failed?5?9?5err?$DN?$CFd?5@ 0000000180006a30     libHeapFilter.obj
 0002:00000a60       ??_C@_0BB@JCNMKLLK@JVMTI_ERROR_NONE@ 0000000180006a60     libHeapFilter.obj
 0002:00000a78       ??_C@_0BL@LDIMKLPH@JVMTI_ERROR_INVALID_THREAD@ 0000000180006a78     libHeapFilter.obj
 0002:00000a98       ??_C@_0CB@PJFPAIKJ@JVMTI_ERROR_INVALID_THREAD_GROU@ 0000000180006a98     libHeapFilter.obj
 0002:00000ac0       ??_C@_0BN@LLMKHMNF@JVMTI_ERROR_INVALID_PRIORITY@ 0000000180006ac0     libHeapFilter.obj
 0002:00000ae0       ??_C@_0CB@MBOFKAGB@JVMTI_ERROR_THREAD_NOT_SUSPENDE@ 0000000180006ae0     libHeapFilter.obj
 0002:00000b08       ??_C@_0BN@FABOLPBI@JVMTI_ERROR_THREAD_SUSPENDED@ 0000000180006b08     libHeapFilter.obj
 0002:00000b28       ??_C@_0BN@FDGNOBJM@JVMTI_ERROR_THREAD_NOT_ALIVE@ 0000000180006b28     libHeapFilter.obj
 0002:00000b48       ??_C@_0BL@GOBIFKNJ@JVMTI_ERROR_INVALID_OBJECT@ 0000000180006b48     libHeapFilter.obj
 0002:00000b68       ??_C@_0BK@FCMAJPPC@JVMTI_ERROR_INVALID_CLASS@ 0000000180006b68     libHeapFilter.obj
 0002:00000b88       ??_C@_0BP@IKLLBKEB@JVMTI_ERROR_CLASS_NOT_PREPARED@ 0000000180006b88     libHeapFilter.obj
 0002:00000ba8       ??_C@_0BN@KLPPLKG@JVMTI_ERROR_INVALID_METHODID@ 0000000180006ba8     libHeapFilter.obj
 0002:00000bc8       ??_C@_0BN@BCEKOKND@JVMTI_ERROR_INVALID_LOCATION@ 0000000180006bc8     libHeapFilter.obj
 0002:00000be8       ??_C@_0BM@DFDGPME@JVMTI_ERROR_INVALID_FIELDID@ 0000000180006be8     libHeapFilter.obj
 0002:00000c08       ??_C@_0BL@NELIEPEC@JVMTI_ERROR_NO_MORE_FRAMES@ 0000000180006c08     libHeapFilter.obj
 0002:00000c28       ??_C@_0BJ@BDBECFDM@JVMTI_ERROR_OPAQUE_FRAME@ 0000000180006c28     libHeapFilter.obj
 0002:00000c48       ??_C@_0BK@MIIFNLOB@JVMTI_ERROR_TYPE_MISMATCH@ 0000000180006c48     libHeapFilter.obj
 0002:00000c68       ??_C@_0BJ@HPCAOILC@JVMTI_ERROR_INVALID_SLOT@ 0000000180006c68     libHeapFilter.obj
 0002:00000c88       ??_C@_0BG@CHILOPNI@JVMTI_ERROR_DUPLICATE@ 0000000180006c88     libHeapFilter.obj
 0002:00000ca0       ??_C@_0BG@DIEMLHKM@JVMTI_ERROR_NOT_FOUND@ 0000000180006ca0     libHeapFilter.obj
 0002:00000cb8       ??_C@_0BM@NHMCKHOB@JVMTI_ERROR_INVALID_MONITOR@ 0000000180006cb8     libHeapFilter.obj
 0002:00000cd8       ??_C@_0BO@PPEDAJGL@JVMTI_ERROR_NOT_MONITOR_OWNER@ 0000000180006cd8     libHeapFilter.obj
 0002:00000cf8       ??_C@_0BG@FCAIPEID@JVMTI_ERROR_INTERRUPT@ 0000000180006cf8     libHeapFilter.obj
 0002:00000d10       ??_C@_0CB@EGDBNKOI@JVMTI_ERROR_INVALID_CLASS_FORMA@ 0000000180006d10     libHeapFilter.obj
 0002:00000d38       ??_C@_0CG@DGKOGIAL@JVMTI_ERROR_CIRCULAR_CLASS_DEFI@ 0000000180006d38     libHeapFilter.obj
 0002:00000d60       ??_C@_0BP@ICEALPKC@JVMTI_ERROR_FAILS_VERIFICATION@ 0000000180006d60     libHeapFilter.obj
 0002:00000d80       ??_C@_0DC@JDACLMIO@JVMTI_ERROR_UNSUPPORTED_REDEFIN@ 0000000180006d80     libHeapFilter.obj
 0002:00000db8       ??_C@_0DE@GKDKNOMJ@JVMTI_ERROR_UNSUPPORTED_REDEFIN@ 0000000180006db8     libHeapFilter.obj
 0002:00000df0       ??_C@_0BO@LAFKIOG@JVMTI_ERROR_INVALID_TYPESTATE@ 0000000180006df0     libHeapFilter.obj
 0002:00000e10       ??_C@_0DH@INDGCLLB@JVMTI_ERROR_UNSUPPORTED_REDEFIN@ 0000000180006e10     libHeapFilter.obj
 0002:00000e48       ??_C@_0DE@NHEOMMGI@JVMTI_ERROR_UNSUPPORTED_REDEFIN@ 0000000180006e48     libHeapFilter.obj
 0002:00000e80       ??_C@_0CA@EKPNJOEP@JVMTI_ERROR_UNSUPPORTED_VERSION@ 0000000180006e80     libHeapFilter.obj
 0002:00000ea0       ??_C@_0BN@OFFMAHHL@JVMTI_ERROR_NAMES_DONT_MATCH@ 0000000180006ea0     libHeapFilter.obj
 0002:00000ec0       ??_C@_0DN@HHBBLAKE@JVMTI_ERROR_UNSUPPORTED_REDEFIN@ 0000000180006ec0     libHeapFilter.obj
 0002:00000f00       ??_C@_0DO@HMBGBGNA@JVMTI_ERROR_UNSUPPORTED_REDEFIN@ 0000000180006f00     libHeapFilter.obj
 0002:00000f40       ??_C@_0BP@PBECGKHJ@JVMTI_ERROR_UNMODIFIABLE_CLASS@ 0000000180006f40     libHeapFilter.obj
 0002:00000f60       ??_C@_0BK@CANILEHF@JVMTI_ERROR_NOT_AVAILABLE@ 0000000180006f60     libHeapFilter.obj
 0002:00000f80       ??_C@_0CE@INJKMEFK@JVMTI_ERROR_MUST_POSSESS_CAPABI@ 0000000180006f80     libHeapFilter.obj
 0002:00000fa8       ??_C@_0BJ@LBFPFPDM@JVMTI_ERROR_NULL_POINTER@ 0000000180006fa8     libHeapFilter.obj
 0002:00000fc8       ??_C@_0BP@CHJPNNEM@JVMTI_ERROR_ABSENT_INFORMATION@ 0000000180006fc8     libHeapFilter.obj
 0002:00000fe8       ??_C@_0BP@OMFMNLC@JVMTI_ERROR_INVALID_EVENT_TYPE@ 0000000180006fe8     libHeapFilter.obj
 0002:00001008       ??_C@_0BN@BIBNPHHO@JVMTI_ERROR_ILLEGAL_ARGUMENT@ 0000000180007008     libHeapFilter.obj
 0002:00001028       ??_C@_0BK@KKNDHDCE@JVMTI_ERROR_NATIVE_METHOD@ 0000000180007028     libHeapFilter.obj
 0002:00001048       ??_C@_0BK@PMKCFHAE@JVMTI_ERROR_OUT_OF_MEMORY@ 0000000180007048     libHeapFilter.obj
 0002:00001068       ??_C@_0BK@NNJBDMNB@JVMTI_ERROR_ACCESS_DENIED@ 0000000180007068     libHeapFilter.obj
 0002:00001088       ??_C@_0BI@GHECLMNC@JVMTI_ERROR_WRONG_PHASE@ 0000000180007088     libHeapFilter.obj
 0002:000010a0       ??_C@_0BF@OLIHJOII@JVMTI_ERROR_INTERNAL@ 00000001800070a0     libHeapFilter.obj
 0002:000010b8       ??_C@_0BO@EOHGKJHI@JVMTI_ERROR_UNATTACHED_THREAD@ 00000001800070b8     libHeapFilter.obj
 0002:000010d8       ??_C@_0CA@LKHFDACL@JVMTI_ERROR_INVALID_ENVIRONMENT@ 00000001800070d8     libHeapFilter.obj
 0002:000010f8       ??_C@_0BA@MMFHLOKK@?$DMunknown?5error?$DO@ 00000001800070f8     libHeapFilter.obj
 0002:00001108       ??_C@_0CF@CBHOKDB@throwable?5?$DN?5jni?9?$DOExceptionOccur@ 0000000180007108     libHeapFilter.obj
 0002:00001130       ??_C@_03OFAPEBGM@?$CFs?6@  0000000180007130     libHeapFilter.obj
 0002:00001138       ??_C@_0DM@LPIGEGNJ@s?2test?2hotspot?2jtreg?2vmTestbase@ 0000000180007138     libHeapFilter.obj
 0002:00001178       ??_C@_0CC@NFCNPEPK@Exception?5in?5JNI?5call?5?$CIcleared?$CJ@ 0000000180007178     libHeapFilter.obj
 0002:000011a0       ??_C@_0BJ@IBAKFIKF@jni?9?$DOExceptionDescribe?$CI?$CJ@ 00000001800071a0     libHeapFilter.obj
 0002:000011c0       ??_C@_0BG@GGKALKMH@jni?9?$DOExceptionClear?$CI?$CJ@ 00000001800071c0     libHeapFilter.obj
 0002:000011d8       ??_C@_0CF@JMGFGJLJ@?$CD?5?5?5verified?5JNI?5assertion?5is?5F@ 00000001800071d8     libHeapFilter.obj
 0002:00001200       ??_C@_07KBAMPNJK@verbose@  0000000180007200     libHeapFilter.obj
 0002:00001208       ??_C@_0DN@PKJBOLAP@nsk_jvmti_parseOptions?$CI?$CJ?3?5unexp@ 0000000180007208     libHeapFilter.obj
 0002:00001248       ??_C@_05IMBNNINJ@trace@    0000000180007248     libHeapFilter.obj
 0002:00001250       ??_C@_0DD@BJKGNDMB@nsk_jvmti_parseOptions?$CI?$CJ?3?5no?5va@ 0000000180007250     libHeapFilter.obj
 0002:00001284       ??_C@_04CGFJFPFD@none@     0000000180007284     libHeapFilter.obj
 0002:0000128c       ??_C@_06BMELKFMA@before@   000000018000728c     libHeapFilter.obj
 0002:00001294       ??_C@_05CMKPCFDK@after@    0000000180007294     libHeapFilter.obj
 0002:0000129c       ??_C@_03NFKEKGGK@all@      000000018000729c     libHeapFilter.obj
 0002:000012a0       ??_C@_0DM@NDNJGJKE@nsk_jvmti_parseOptions?$CI?$CJ?3?5uexpe@ 00000001800072a0     libHeapFilter.obj
 0002:000012e0       ??_C@_08NBBJKJO@waittime@  00000001800072e0     libHeapFilter.obj
 0002:000012f0       ??_C@_0DO@CMHGAOHC@nsk_jvmti_parseOptions?$CI?$CJ?3?5not?5i@ 00000001800072f0     libHeapFilter.obj
 0002:00001330       ??_C@_0DL@LNMPBDLN@nsk_jvmti_parseOptions?$CI?$CJ?3?5negat@ 0000000180007330     libHeapFilter.obj
 0002:00001370       ??_C@_0DA@GMFJNOJH@nsk_jvmti_parseOptions?$CI?$CJ?3?5unkno@ 0000000180007370     libHeapFilter.obj
 0002:000013a0       ??_C@_0CO@CCIAMEAN@nsk_jvmti_parseOptions?$CI?$CJ?3?5found@ 00000001800073a0     libHeapFilter.obj
 0002:000013d0       ??_C@_0CJ@OEGPCGDL@nsk_jvmti_parseOptions?$CI?$CJ?3?5out?5o@ 00000001800073d0     libHeapFilter.obj
 0002:00001400       ??_C@_0DI@NMBHPGGF@nsk_jvmti_parseOptions?$CI?$CJ?3?5too?5m@ 0000000180007400     libHeapFilter.obj
 0002:00001438       ??_C@_03POGCGECB@?5?0?$HO@ 0000000180007438     libHeapFilter.obj
 0002:00001440       ??_C@_0DC@GKLNPJIJ@nsk_jvmti_findOptionValue?$CI?$CJ?3?5op@ 0000000180007440     libHeapFilter.obj
 0002:00001478       ??_C@_0CB@MLNJNCLJ@?5?5jvmti?5error?3?5code?$DN?$CFd?0?5name?$DN?$CFs@ 0000000180007478     libHeapFilter.obj
 0002:000014a0       ??_C@_0CD@OHBGDKMK@?$CD?5?5?5jvmti?5error?3?5code?$DN?$CFd?0?5name?$DN@ 00000001800074a0     libHeapFilter.obj
 0002:000014c8       ??_C@_0CG@JNNCGPHB@?$CD?5?5?5error?5expected?3?5code?$DN?$CFd?0?5na@ 00000001800074c8     libHeapFilter.obj
 0002:000014f0       ??_C@_0EB@IMGKPCGE@?$CIstr_obj?5?$DN?5jni?9?$DONewStringUTF?$CIco@ 00000001800074f0     libHeapFilter.obj
 0002:00001540       ??_C@_0EA@HFOGGBCC@s?2test?2hotspot?2jtreg?2vmTestbase@ 0000000180007540     libHeapFilter.obj
 0002:00001580       ??_C@_05KKCIMGE@error@     0000000180007580     libHeapFilter.obj
 0002:00001588       ??_C@_0CJ@JACLEAA@Test?5failed?5by?5setFailStatus?$CI?$CJ?4@ 0000000180007588     libHeapFilter.obj
 0002:000015b8       ??_C@_0BD@HGNAOMCP@agent_data_monitor@ 00000001800075b8     libHeapFilter.obj
 0002:000015d0       ??_C@_0EB@OGCLGKLN@javaVM?9?$DOGetEnv?$CI?$CIvoid?5?$CK?$CK?$CJ?$CGjvmti_@ 00000001800075d0     libHeapFilter.obj
 0002:00001620       ??_C@_0EA@PNBCDMOA@s?2test?2hotspot?2jtreg?2vmTestbase@ 0000000180007620     libHeapFilter.obj
 0002:00001660       ??_C@_0CI@DDPIFBGM@init_agent_data?$CIjvmti_env?0?5?$CGage@ 0000000180007660     libHeapFilter.obj
 0002:00001688       ??_C@_0DI@ILAHDLMP@?$CI?$CKagentThreadProc?$CJ?$CIjvmti_env?0?5a@ 0000000180007688     libHeapFilter.obj
 0002:000016c0       ??_C@_0BD@KDBALNLB@JVMTI?5agent?5thread@ 00000001800076c0     libHeapFilter.obj
 0002:000016d8       ??_C@_0BB@NOKBFPFO@java?1lang?1Thread@ 00000001800076d8     libHeapFilter.obj
 0002:000016ec       ??_C@_06FALKBLGB@?$DMinit?$DO@ 00000001800076ec     libHeapFilter.obj
 0002:000016f8       ??_C@_0BG@IKDDPPGD@?$CILjava?1lang?1String?$DL?$CJV@ 00000001800076f8     libHeapFilter.obj
 0002:00001710       ??_C@_0EB@IFJBFEKC@?$CIthreadClass?5?$DN?5jni_env?9?$DOFindCla@ 0000000180007710     libHeapFilter.obj
 0002:00001760       ??_C@_0GF@FGFIBKKL@?$CIthreadCtor?5?$DN?5jni_env?9?$DOGetMetho@ 0000000180007760     libHeapFilter.obj
 0002:000017c8       ??_C@_0DN@NCPDJLOG@?$CIthreadName?5?$DN?5jni_env?9?$DONewStrin@ 00000001800077c8     libHeapFilter.obj
 0002:00001810       ??_C@_0FE@PFKODBGC@?$CIthreadObject?5?$DN?5jni_env?9?$DONewObj@ 0000000180007810     libHeapFilter.obj
 0002:00001870       ??_C@_0ED@HOBAHHJI@?$CIthreadGlobalRef?5?$DN?5jni_env?9?$DONew@ 0000000180007870     libHeapFilter.obj
 0002:000018c0       ??_C@_0FN@HNJJAHFC@jvmti_env?9?$DORunAgentThread?$CIagent@ 00000001800078c0     libHeapFilter.obj
 0002:00001920       ??_C@_0EA@MOJDNKDF@Debuggee?5status?5sync?5aborted?5be@ 0000000180007920     libHeapFilter.obj
 0002:00001960       ??_C@_0CO@PGPGMHBJ@No?5status?5sync?5occured?5for?5time@ 0000000180007960     libHeapFilter.obj
 0002:00001990       ??_C@_0CL@DOEBDPKJ@Debuggee?5was?5not?5suspended?5on?5s@ 0000000180007990     libHeapFilter.obj
 0002:000019c0       ??_C@_0EA@EEOEJAEN@status?5?$DN?5syncDebuggeeStatus?$CIjni@ 00000001800079c0     libHeapFilter.obj
 0002:00001a00       ??_C@_0BL@JBCFNBMB@nsk_jvmti_resetAgentData?$CI?$CJ@ 0000000180007a00     libHeapFilter.obj
 0002:00001a20       ??_C@_0DN@NNGECJON@jvmti_env?9?$DOSetEventNotification@ 0000000180007a20     libHeapFilter.obj
 0002:00001a60       ??_C@_0EL@LPBEELIP@s?2test?2hotspot?2jtreg?2vmTestbase@ 0000000180007a60     libHeapFilter.obj
 0002:00001ab0       ??_C@_0CK@JDAMFDMJ@jvmti?9?$DOSetTag?$CIo?0?5tag?$CJ?5?$DN?$DN?5JVMTI_@ 0000000180007ab0     libHeapFilter.obj
 0002:00001ae0       ??_C@_0CC@DAMNHKNI@Can?8t?5set?5tag?5?$CFli?5for?5object?5?$CFl@ 0000000180007ae0     libHeapFilter.obj
 0002:00001b08       ??_C@_0DL@HAJPNKEF@jvmti?9?$DOGetObjectHashCode?$CIo?0?5?$CGha@ 0000000180007b08     libHeapFilter.obj
 0002:00001b48       ??_C@_0BL@JFPIEOBF@Can?8t?5get?5hash?5object?5?$CFlx?6@ 0000000180007b48     libHeapFilter.obj
 0002:00001b68       ??_C@_0BG@DICPHBKN@setTag?3?5?$CF08x?5?$DM?9?5?$CF?53li@ 0000000180007b68     libHeapFilter.obj
 0002:00001b80       ??_C@_0DH@FCEEBDMJ@?$CIs?5?$DN?5jni?9?$DOGetStringUTFChars?$CIsIn@ 0000000180007b80     libHeapFilter.obj
 0002:00001bb8       ??_C@_0BJ@OKKGHDCN@Can?8t?5get?5string?5at?5?$CF?$CDp?6@ 0000000180007bb8     libHeapFilter.obj
 0002:00001bd8       ??_C@_0BP@EKFLGGFJ@Can?8t?5get?5string?5at?5?$CF?$CDp?3?5null?6@ 0000000180007bd8     libHeapFilter.obj
 0002:00001bf8       ??_C@_06ICODBHCL@?5?1?1?5?$CFs@ 0000000180007bf8     libHeapFilter.obj
 0002:00001c00       ??_C@_0DB@KGFPLEGO@?$CIr?5?$DN?5jvmti?9?$DOGetTag?$CIo?0?5?$CGtag?$CJ?$CJ?5?$DN?$DN@ 0000000180007c00     libHeapFilter.obj
 0002:00001c38       ??_C@_0CO@PDAGBCGJ@Can?8t?5GetTag?5for?5object?5?$CFlx?4?5Re@ 0000000180007c38     libHeapFilter.obj
 0002:00001c68       ??_C@_0CH@HPEODOHC@TEST_BUG?3?5Max?4?5number?5of?5refs?5r@ 0000000180007c68     libHeapFilter.obj
 0002:00001c90       ??_C@_0DI@PHFCABIM@?$CIr?5?$DN?5jvmti?9?$DOGetTag?$CIfrom?0?5?$CGtagFr@ 0000000180007c90     libHeapFilter.obj
 0002:00001cc8       ??_C@_0DI@MDEGFNKD@TEST_BUG?3?5Can?8t?5GetTag?5for?5obje@ 0000000180007cc8     libHeapFilter.obj
 0002:00001d00       ??_C@_0DE@MLELJAHM@?$CIr?5?$DN?5jvmti?9?$DOGetTag?$CIto?0?5?$CGtagTo?$CJ?$CJ@ 0000000180007d00     libHeapFilter.obj
 0002:00001d34       ??_C@_01GFHCPBMG@C@        0000000180007d34     libHeapFilter.obj
 0002:00001d38       ??_C@_01HMGJMAIH@B@        0000000180007d38     libHeapFilter.obj
 0002:00001d3c       ??_C@_01CPLAODJH@S@        0000000180007d3c     libHeapFilter.obj
 0002:00001d40       ??_C@_01JPJNBJEM@I@        0000000180007d40     libHeapFilter.obj
 0002:00001d44       ??_C@_01LELAEKIP@J@        0000000180007d44     libHeapFilter.obj
 0002:00001d48       ??_C@_01BIAFAFID@F@        0000000180007d48     libHeapFilter.obj
 0002:00001d4c       ??_C@_01CKDDGHAB@D@        0000000180007d4c     libHeapFilter.obj
 0002:00001d50       ??_C@_01POHCFINO@Z@        0000000180007d50     libHeapFilter.obj
 0002:00001d58       ??_C@_0CO@GDAFHICB@verify_tag?$CIobject_class_tag?0?5?$CKo@ 0000000180007d58     libHeapFilter.obj
 0002:00001d90       ??_C@_0FK@GEODHOED@s?2test?2hotspot?2jtreg?2vmTestbase@ 0000000180007d90     libHeapFilter.obj
 0002:00001df0       ??_C@_0CA@JHENKMMM@verify_tag?$CIclass_tag?0?5?$CKtag_ptr?$CJ@ 0000000180007df0     libHeapFilter.obj
 0002:00001e10       ??_C@_0FI@KDHDLMAD@Tag?5values?5invalid?5for?5selected@ 0000000180007e10     libHeapFilter.obj
 0002:00001e68       ??_C@_0CI@BKHIAJGL@?7Class?5tag?3?50x?$CFlX?$DL?6?7Object?5tag?3@ 0000000180007e68     libHeapFilter.obj
 0002:00001e90       ??_C@_0BD@JFADHEFE@Ljava?1lang?1String?$DL@ 0000000180007e90     libHeapFilter.obj
 0002:00001ea4       ??_C@_02EBOMBDPA@?$FLI@    0000000180007ea4     libHeapFilter.obj
 0002:00001ea8       ??_C@_0DB@PCFPGDFE@nullptr?5?$CB?$DN?5?$CIdebugee?5?$DN?5jni?9?$DOFind@ 0000000180007ea8     libHeapFilter.obj
 0002:00001ee0       ??_C@_0DG@LBICOMJD@nsk?1jvmti?1IterateThroughHeap?1fi@ 0000000180007ee0     libHeapFilter.obj
 0002:00001f20       ??_C@_0FE@CJLNEJIL@nullptr?5?$CB?$DN?5?$CItestObjectsField?5?$DN?5@ 0000000180007f20     libHeapFilter.obj
 0002:00001f78       ??_C@_0BE@EOPHJDGO@?$FLLjava?1lang?1Object?$DL@ 0000000180007f78     libHeapFilter.obj
 0002:00001f90       ??_C@_0M@FIIEPOPL@testObjects@ 0000000180007f90     libHeapFilter.obj
 0002:00001fa0       ??_C@_0GB@OOHNFBFO@nullptr?5?$CB?$DN?5?$CItestObjects?5?$DN?5?$CIjobj@ 0000000180007fa0     libHeapFilter.obj
 0002:00002010       ??_C@_0EG@EGKECOCG@nullptr?5?$CB?$DN?5?$CItarget?5?$DN?5jni?9?$DOGetOb@ 0000000180008010     libHeapFilter.obj
 0002:00002058       ??_C@_0DH@MGPEEDOG@nullptr?5?$CB?$DN?5?$CItargetClass?5?$DN?5jni?9?$DO@ 0000000180008058     libHeapFilter.obj
 0002:00002090       ??_C@_0EN@PENBOMLE@jvmti?9?$DOGetClassSignature?$CItarget@ 0000000180008090     libHeapFilter.obj
 0002:000020e0       ??_C@_0FJ@EJDGOBIL@jvmti?9?$DOGetClassFields?$CI?5targetCl@ 00000001800080e0     libHeapFilter.obj
 0002:00002140       ??_C@_0JI@INPGDKIP@jvmti?9?$DOGetFieldName?$CItargetClass@ 0000000180008140     libHeapFilter.obj
 0002:000021e0       ??_C@_0EI@BJHKIOL@jvmti?9?$DOGetFieldModifiers?$CI?5targe@ 00000001800081e0     libHeapFilter.obj
 0002:00002230       ??_C@_0FC@NCIFDNEJ@nullptr?5?$CB?$DN?5?$CIvalue?5?$DN?5jni?9?$DOGetSta@ 0000000180008230     libHeapFilter.obj
 0002:00002290       ??_C@_0EG@OFDEFKIK@nullptr?5?$CB?$DN?5?$CIvalue?5?$DN?5jni?9?$DOGetObj@ 0000000180008290     libHeapFilter.obj
 0002:000022d8       ??_C@_0DJ@ONJGBKOM@jvmti?9?$DOSetTag?$CIvalue?0?5ENCODE_TAG@ 00000001800082d8     libHeapFilter.obj
 0002:00002318       ??_C@_0DH@LMCGIBGC@jvmti?9?$DOSetTag?$CItarget?0?5ENCODE_TA@ 0000000180008318     libHeapFilter.obj
 0002:00002350       ??_C@_0DL@JLFJEFJO@jvmti?9?$DOSetTag?$CItargetClass?0?5ENCO@ 0000000180008350     libHeapFilter.obj
 0002:00002390       ??_C@_0DA@OPPCAIO@jvmti?9?$DODeallocate?$CI?$CIunsigned?5cha@ 0000000180008390     libHeapFilter.obj
 0002:000023c0       ??_C@_0EI@FDMBNFHF@Field?5?$CFs?3?3?$CFs?5expected?5to?5be?5fou@ 00000001800083c0     libHeapFilter.obj
 0002:00002408       ??_C@_0BC@BPPEGBIH@Waiting?5debugee?4?6@ 0000000180008408     libHeapFilter.obj
 0002:00002420       ??_C@_0DJ@GDOKODHN@nsk_jvmti_enableEvents?$CIJVMTI_EN@ 0000000180008420     libHeapFilter.obj
 0002:00002460       ??_C@_0BP@LAIJOMPC@nsk_jvmti_waitForSync?$CItimeout?$CJ@ 0000000180008460     libHeapFilter.obj
 0002:00002480       ??_C@_0BB@ENNPPLIL@Tagging?5fields?4?6@ 0000000180008480     libHeapFilter.obj
 0002:00002498       ??_C@_0CC@HNDBEALC@JNI_OK?5?$DN?$DN?5tag_objects?$CIjvmti?0?5jn@ 0000000180008498     libHeapFilter.obj
 0002:000024c0       ??_C@_0CD@IPANCNID@Iterating?5over?5reachable?5object@ 00000001800084c0     libHeapFilter.obj
 0002:000024f0       ??_C@_0EP@JMNGKNDM@jvmti?9?$DOIterateThroughHeap?$CIfilte@ 00000001800084f0     libHeapFilter.obj
 0002:00002540       ??_C@_0CH@BAIMKILI@Verifying?5that?5all?5fields?5were?5@ 0000000180008540     libHeapFilter.obj
 0002:00002568       ??_C@_0BH@LECMGIIA@nsk_jvmti_resumeSync?$CI?$CJ@ 0000000180008568     libHeapFilter.obj
 0002:00002580       ??_C@_0CF@ENEMFJFH@Iterating?5over?5unreachable?5obje@ 0000000180008580     libHeapFilter.obj
 0002:000025b0       ??_C@_0EI@OBBECNBE@jvmti?9?$DOSetEventCallbacks?$CI?$CGevent@ 00000001800085b0     libHeapFilter.obj
 0002:000025f8       ??_C@_0BB@CGPOECH@jvmti?5?$CB?$DN?5nullptr@ 00000001800085f8     libHeapFilter.obj
 0002:0000260c       ??_C@_06EOIELIPE@filter@   000000018000860c     libHeapFilter.obj
 0002:00002618       ??_C@_0BJ@KHDGPMAG@JVMTI_HEAP_FILTER_TAGGED@ 0000000180008618     libHeapFilter.obj
 0002:00002638       ??_C@_0BL@CGFEOEIC@JVMTI_HEAP_FILTER_UNTAGGED@ 0000000180008638     libHeapFilter.obj
 0002:00002658       ??_C@_0BP@CAAANLHI@JVMTI_HEAP_FILTER_CLASS_TAGGED@ 0000000180008658     libHeapFilter.obj
 0002:00002678       ??_C@_0CB@DCOCICKH@JVMTI_HEAP_FILTER_CLASS_UNTAGGE@ 0000000180008678     libHeapFilter.obj
 0002:000026a0       ??_C@_0BM@GFMLBADL@unknown?5filter?5value?5?8?$CFs?8?4?6@ 00000001800086a0     libHeapFilter.obj
 0002:000026c0       ??_C@_0CE@FILIJFML@filter?5option?5shound?5be?5present@ 00000001800086c0     libHeapFilter.obj
 0002:000026e8       ??_C@_0BO@DBKDIPGD@jvmti?9?$DOAddCapabilities?$CI?$CGcaps?$CJ@ 00000001800086e8     libHeapFilter.obj
 0002:00002708       ??_C@_0CH@MPLODCED@nsk_jvmti_setAgentProc?$CIagent?0?5n@ 0000000180008708     libHeapFilter.obj
 0002:00002740       ??_C@_1EC@JIJBPKFM@?$AAa?$AAp?$AAi?$AA?9?$AAm?$AAs?$AA?9?$AAw?$AAi?$AAn?$AA?9?$AAc?$AAo?$AAr?$AAe@ 0000000180008740     MSVCRT:thread_safe_statics.obj
 0002:00002788       ??_C@_1BK@MGMFAEKH@?$AAk?$AAe?$AAr?$AAn?$AAe?$AAl?$AA3?$AA2?$AA?4?$AAd?$AAl?$AAl@ 0000000180008788     MSVCRT:thread_safe_statics.obj
 0002:000027a8       ??_C@_0BJ@JEBJOJFJ@SleepConditionVariableCS@ 00000001800087a8     MSVCRT:thread_safe_statics.obj
 0002:000027c8       ??_C@_0BJ@PGPPEPCC@WakeAllConditionVariable@ 00000001800087c8     MSVCRT:thread_safe_statics.obj
 0002:000027e8       _pDefaultRawDllMain        00000001800087e8     MSVCRT:dll_dllmain.obj
 0002:000027e8       _pRawDllMain               00000001800087e8     MSVCRT:dll_dllmain.obj
 0002:000027f0       __xmm@ffffffffffffffffffffffffffffffff 00000001800087f0     MSVCRT:utility.obj
 0002:00002800       _load_config_used          0000000180008800     MSVCRT:loadcfg.obj
 0002:00002a00       _tls_used                  0000000180008a00     MSVCRT:tlssup.obj
 0002:00002a28       __volatile_metadata        0000000180008a28     <linker-defined>
 0002:00002e28       __rtc_iaa                  0000000180008e28     MSVCRT:initsect.obj
 0002:00002e30       __rtc_izz                  0000000180008e30     MSVCRT:initsect.obj
 0002:00002e38       __rtc_taa                  0000000180008e38     MSVCRT:initsect.obj
 0002:00002e40       __rtc_tzz                  0000000180008e40     MSVCRT:initsect.obj
 0002:00002e48       _tls_start                 0000000180008e48     MSVCRT:tlssup.obj
 0002:00002e4c       _Init_thread_epoch         0000000180008e4c     MSVCRT:thread_safe_statics.obj
 0002:00002e50       _tls_end                   0000000180008e50     MSVCRT:tlssup.obj
 0002:000035a4       __IMPORT_DESCRIPTOR_KERNEL32 00000001800095a4     kernel32:KERNEL32.dll
 0002:000035b8       __IMPORT_DESCRIPTOR_VCRUNTIME140 00000001800095b8     vcruntime:VCRUNTIME140.dll
 0002:000035cc       __IMPORT_DESCRIPTOR_api-ms-win-crt-heap-l1-1-0 00000001800095cc     ucrt:api-ms-win-crt-heap-l1-1-0.dll
 0002:000035e0       __IMPORT_DESCRIPTOR_api-ms-win-crt-runtime-l1-1-0 00000001800095e0     ucrt:api-ms-win-crt-runtime-l1-1-0.dll
 0002:000035f4       __IMPORT_DESCRIPTOR_api-ms-win-crt-convert-l1-1-0 00000001800095f4     ucrt:api-ms-win-crt-convert-l1-1-0.dll
 0002:00003608       __IMPORT_DESCRIPTOR_api-ms-win-crt-stdio-l1-1-0 0000000180009608     ucrt:api-ms-win-crt-stdio-l1-1-0.dll
 0002:0000361c       __IMPORT_DESCRIPTOR_api-ms-win-crt-string-l1-1-0 000000018000961c     ucrt:api-ms-win-crt-string-l1-1-0.dll
 0002:00003630       __NULL_IMPORT_DESCRIPTOR   0000000180009630     kernel32:KERNEL32.dll
 0003:00000060       _Init_global_epoch         000000018000a060     MSVCRT:thread_safe_statics.obj
 0003:00000070       __security_cookie          000000018000a070     MSVCRT:gs_cookie.obj
 0003:00000078       __security_cookie_complement 000000018000a078     MSVCRT:gs_cookie.obj
 0003:00000080       __scrt_native_dllmain_reason 000000018000a080     MSVCRT:utility.obj
 0003:00000088       __isa_available            000000018000a088     MSVCRT:cpu_disp.obj
 0003:0000008c       __isa_enabled              000000018000a08c     MSVCRT:cpu_disp.obj
 0003:00000090       __memset_fast_string_threshold 000000018000a090     MSVCRT:cpu_disp.obj
 0003:00000098       __memset_nt_threshold      000000018000a098     MSVCRT:cpu_disp.obj
 0003:000000a0       __scrt_ucrt_dll_is_in_use  000000018000a0a0     MSVCRT:ucrt_stubs.obj
 0003:000000b0       g_wrongHeapCallbacks       000000018000a0b0     libHeapFilter.obj
 0003:00000130       g_szTagInfo                000000018000a130     libHeapFilter.obj
 0003:00002070       g_tagFlags                 000000018000c070     libHeapFilter.obj
 0003:00002458       g_refsToVerifyCnt          000000018000c458     libHeapFilter.obj
 0003:0000245c       g_fakeUserData             000000018000c45c     libHeapFilter.obj
 0003:00002460       g_tagVisitCount            000000018000c460     libHeapFilter.obj
 0003:00003400       g_refsToVerify             000000018000d400     libHeapFilter.obj
 0003:0001ab00       g_userDataError            0000000180024b00     libHeapFilter.obj
 0003:0001acf0       ?_OptionsStorage@?1??__local_stdio_printf_options@@9@4_KA 0000000180024cf0     libHeapFilter.obj
 0003:0001b2b8       _tls_index                 00000001800252b8     MSVCRT:tlssup.obj
 0003:0001b2c0       __scrt_current_native_startup_state 00000001800252c0     MSVCRT:utility.obj
 0003:0001b2c8       __scrt_native_startup_lock 00000001800252c8     MSVCRT:utility.obj
 0003:0001b308       __scrt_debugger_hook_flag  0000000180025308     MSVCRT:utility_desktop.obj
 0003:0001b310       ?__type_info_root_node@@3U__type_info_node@@A 0000000180025310     MSVCRT:tncleanup.obj
 0003:0001b320       ?_OptionsStorage@?1??__local_stdio_scanf_options@@9@4_KA 0000000180025320     MSVCRT:default_local_stdio_options.obj
 0003:0001b328       __favor                    0000000180025328     MSVCRT:cpu_disp.obj
 0003:0001b330       __dyn_tls_init_callback    0000000180025330     <common>

 entry point at        0001:00004210

 Static symbols

 0000:fffd8000       .debug$S                   0000000180000000     HeapFilter.exp
 0000:fffd8000       .debug$S                   0000000180000000     vcruntime:VCRUNTIME140.dll
 0000:fffd8000       .debug$S                   0000000180000000     vcruntime:VCRUNTIME140.dll
 0000:fffd8000       .debug$S                   0000000180000000     vcruntime:VCRUNTIME140.dll
 0000:fffd8000       .debug$S                   0000000180000000     vcruntime:VCRUNTIME140.dll
 0000:fffd8000       .debug$S                   0000000180000000     vcruntime:VCRUNTIME140.dll
 0000:fffd8000       .debug$S                   0000000180000000     vcruntime:VCRUNTIME140.dll
 0000:fffd8000       .debug$S                   0000000180000000     vcruntime:VCRUNTIME140.dll
 0000:fffd8000       .debug$S                   0000000180000000     ucrt:api-ms-win-crt-convert-l1-1-0.dll
 0000:fffd8000       .debug$S                   0000000180000000     ucrt:api-ms-win-crt-heap-l1-1-0.dll
 0000:fffd8000       .debug$S                   0000000180000000     ucrt:api-ms-win-crt-heap-l1-1-0.dll
 0000:fffd8000       .debug$S                   0000000180000000     ucrt:api-ms-win-crt-heap-l1-1-0.dll
 0000:fffd8000       .debug$S                   0000000180000000     ucrt:api-ms-win-crt-heap-l1-1-0.dll
 0000:fffd8000       .debug$S                   0000000180000000     ucrt:api-ms-win-crt-runtime-l1-1-0.dll
 0000:fffd8000       .debug$S                   0000000180000000     ucrt:api-ms-win-crt-runtime-l1-1-0.dll
 0000:fffd8000       .debug$S                   0000000180000000     ucrt:api-ms-win-crt-runtime-l1-1-0.dll
 0000:fffd8000       .debug$S                   0000000180000000     ucrt:api-ms-win-crt-runtime-l1-1-0.dll
 0000:fffd8000       .debug$S                   0000000180000000     ucrt:api-ms-win-crt-runtime-l1-1-0.dll
 0000:fffd8000       .debug$S                   0000000180000000     ucrt:api-ms-win-crt-runtime-l1-1-0.dll
 0000:fffd8000       .debug$S                   0000000180000000     ucrt:api-ms-win-crt-runtime-l1-1-0.dll
 0000:fffd8000       .debug$S                   0000000180000000     ucrt:api-ms-win-crt-runtime-l1-1-0.dll
 0000:fffd8000       .debug$S                   0000000180000000     ucrt:api-ms-win-crt-runtime-l1-1-0.dll
 0000:fffd8000       .debug$S                   0000000180000000     ucrt:api-ms-win-crt-runtime-l1-1-0.dll
 0000:fffd8000       .debug$S                   0000000180000000     ucrt:api-ms-win-crt-runtime-l1-1-0.dll
 0000:fffd8000       .debug$S                   0000000180000000     ucrt:api-ms-win-crt-runtime-l1-1-0.dll
 0000:fffd8000       .debug$S                   0000000180000000     ucrt:api-ms-win-crt-runtime-l1-1-0.dll
 0000:fffd8000       .debug$S                   0000000180000000     ucrt:api-ms-win-crt-runtime-l1-1-0.dll
 0000:fffd8000       .debug$S                   0000000180000000     ucrt:api-ms-win-crt-runtime-l1-1-0.dll
 0000:fffd8000       .debug$S                   0000000180000000     ucrt:api-ms-win-crt-runtime-l1-1-0.dll
 0000:fffd8000       .debug$S                   0000000180000000     ucrt:api-ms-win-crt-stdio-l1-1-0.dll
 0000:fffd8000       .debug$S                   0000000180000000     ucrt:api-ms-win-crt-stdio-l1-1-0.dll
 0000:fffd8000       .debug$S                   0000000180000000     ucrt:api-ms-win-crt-stdio-l1-1-0.dll
 0000:fffd8000       .debug$S                   0000000180000000     ucrt:api-ms-win-crt-stdio-l1-1-0.dll
 0000:fffd8000       .debug$S                   0000000180000000     ucrt:api-ms-win-crt-stdio-l1-1-0.dll
 0000:fffd8000       .debug$S                   0000000180000000     ucrt:api-ms-win-crt-stdio-l1-1-0.dll
 0000:fffd8000       .debug$S                   0000000180000000     ucrt:api-ms-win-crt-stdio-l1-1-0.dll
 0000:fffd8000       .debug$S                   0000000180000000     ucrt:api-ms-win-crt-stdio-l1-1-0.dll
 0000:fffd8000       .debug$S                   0000000180000000     ucrt:api-ms-win-crt-stdio-l1-1-0.dll
 0000:fffd8000       .debug$S                   0000000180000000     ucrt:api-ms-win-crt-stdio-l1-1-0.dll
 0000:fffd8000       .debug$S                   0000000180000000     ucrt:api-ms-win-crt-string-l1-1-0.dll
 0000:fffd8000       .debug$S                   0000000180000000     ucrt:api-ms-win-crt-string-l1-1-0.dll
 0000:fffd8000       .debug$S                   0000000180000000     ucrt:api-ms-win-crt-string-l1-1-0.dll
 0000:fffd8000       .debug$S                   0000000180000000     ucrt:api-ms-win-crt-string-l1-1-0.dll
 0000:fffd8000       .debug$S                   0000000180000000     ucrt:api-ms-win-crt-string-l1-1-0.dll
 0000:fffd8000       .debug$S                   0000000180000000     ucrt:api-ms-win-crt-string-l1-1-0.dll
 0000:fffd8000       .debug$S                   0000000180000000     ucrt:api-ms-win-crt-string-l1-1-0.dll
 0000:fffd8000       .debug$S                   0000000180000000     ucrt:api-ms-win-crt-string-l1-1-0.dll
 0000:fffd8000       .debug$S                   0000000180000000     ucrt:api-ms-win-crt-string-l1-1-0.dll
 0000:fffd8000       .debug$S                   0000000180000000     kernel32:KERNEL32.dll
 0000:fffd8000       .debug$S                   0000000180000000     kernel32:KERNEL32.dll
 0000:fffd8000       .debug$S                   0000000180000000     kernel32:KERNEL32.dll
 0000:fffd8000       .debug$S                   0000000180000000     kernel32:KERNEL32.dll
 0000:fffd8000       .debug$S                   0000000180000000     kernel32:KERNEL32.dll
 0000:fffd8000       .debug$S                   0000000180000000     kernel32:KERNEL32.dll
 0000:fffd8000       .debug$S                   0000000180000000     kernel32:KERNEL32.dll
 0000:fffd8000       .debug$S                   0000000180000000     kernel32:KERNEL32.dll
 0000:fffd8000       .debug$S                   0000000180000000     kernel32:KERNEL32.dll
 0000:fffd8000       .debug$S                   0000000180000000     kernel32:KERNEL32.dll
 0000:fffd8000       .debug$S                   0000000180000000     kernel32:KERNEL32.dll
 0000:fffd8000       .debug$S                   0000000180000000     kernel32:KERNEL32.dll
 0000:fffd8000       .debug$S                   0000000180000000     kernel32:KERNEL32.dll
 0000:fffd8000       .debug$S                   0000000180000000     kernel32:KERNEL32.dll
 0000:fffd8000       .debug$S                   0000000180000000     kernel32:KERNEL32.dll
 0000:fffd8000       .debug$S                   0000000180000000     kernel32:KERNEL32.dll
 0000:fffd8000       .debug$S                   0000000180000000     kernel32:KERNEL32.dll
 0000:fffd8000       .debug$S                   0000000180000000     kernel32:KERNEL32.dll
 0000:fffd8000       .debug$S                   0000000180000000     kernel32:KERNEL32.dll
 0000:fffd8000       .debug$S                   0000000180000000     kernel32:KERNEL32.dll
 0000:fffd8000       .debug$S                   0000000180000000     kernel32:KERNEL32.dll
 0000:fffd8000       .debug$S                   0000000180000000     kernel32:KERNEL32.dll
 0000:fffd8000       .debug$S                   0000000180000000     kernel32:KERNEL32.dll
 0000:fffd8000       .debug$S                   0000000180000000     kernel32:KERNEL32.dll
 0000:fffd8000       .debug$S                   0000000180000000     kernel32:KERNEL32.dll
 0000:fffd8000       .debug$S                   0000000180000000     kernel32:KERNEL32.dll
 0000:fffd8000       .debug$S                   0000000180000000     kernel32:KERNEL32.dll
 0000:fffd8000       .debug$S                   0000000180000000     kernel32:KERNEL32.dll
 0001:00000000       ??__ETAGGED_INT_VALUE@@YAXXZ 0000000180001000 f   libHeapFilter.obj
 0001:00000014       ??__ETAGGED_STATIC_INT_VALUE@@YAXXZ 0000000180001014 f   libHeapFilter.obj
 0001:00000028       ??__EUNTAGGED_INT_VALUE@@YAXXZ 0000000180001028 f   libHeapFilter.obj
 0001:0000003c       ??__EUNTAGGED_STATIC_INT_VALUE@@YAXXZ 000000018000103c f   libHeapFilter.obj
 0001:00000fb8       addRefToVerify             0000000180001fb8 f   libHeapFilter.obj
 0001:00001024       agent                      0000000180002024 f   libHeapFilter.obj
 0001:00001484       agentThreadWrapper         0000000180002484 f   libHeapFilter.obj
 0001:00001710       check_option               0000000180002710 f   libHeapFilter.obj
 0001:00001a38       file_basename              0000000180002a38 f   libHeapFilter.obj
 0001:00002aec       startAgentThreadWrapper    0000000180003aec f   libHeapFilter.obj
 0001:00002f54       syncDebuggeeStatus         0000000180003f54 f   libHeapFilter.obj
 0001:00003cd4       capture_previous_context   0000000180004cd4 f   MSVCRT:gs_report.obj
 0001:00003d48       ?__scrt_initialize_thread_safe_statics@@YAHXZ 0000000180004d48 f   MSVCRT:thread_safe_statics.obj
 0001:00003e18       ?__scrt_uninitialize_thread_safe_statics@@YAXXZ 0000000180004e18 f   MSVCRT:thread_safe_statics.obj
 0001:00003ec0       $$000000                   0000000180004ec0     MSVCRT:amdsecgs.obj
 0001:00003ef0       ?dllmain_crt_dispatch@@YAHQEAUHINSTANCE__@@KQEAX@Z 0000000180004ef0 f   MSVCRT:dll_dllmain.obj
 0001:00003f40       ?dllmain_crt_process_attach@@YAHQEAUHINSTANCE__@@QEAX@Z 0000000180004f40 f   MSVCRT:dll_dllmain.obj
 0001:00004058       ?dllmain_crt_process_detach@@YAH_N@Z 0000000180005058 f   MSVCRT:dll_dllmain.obj
 0001:000040dc       ?dllmain_dispatch@@YAHQEAUHINSTANCE__@@KQEAX@Z 00000001800050dc f   MSVCRT:dll_dllmain.obj
 0001:00004af0       $$000000                   0000000180005af0     MSVCRT:guard_dispatch.obj
 0001:00004b10       $$000000                   0000000180005b10     MSVCRT:guard_xfg_dispatch.obj
 0001:00004b26       ?fin$0@?0??dllmain_crt_process_attach@@YAHQEAUHINSTANCE__@@QEAX@Z@4HA 0000000180005b26 f   MSVCRT:dll_dllmain.obj
 0001:00004b3d       ?fin$0@?0??dllmain_crt_process_detach@@YAH_N@Z@4HA 0000000180005b3d f   MSVCRT:dll_dllmain.obj
 0001:00004b56       ?fin$1@?0??dllmain_crt_process_detach@@YAH_N@Z@4HA 0000000180005b56 f   MSVCRT:dll_dllmain.obj
 0001:00004b6a       ?filt$0@?0??dllmain_dispatch@@YAHQEAUHINSTANCE__@@KQEAX@Z@4HA 0000000180005b6a f   MSVCRT:dll_dllmain.obj
 0001:00004ba0       __scrt_is_nonwritable_in_current_image$filt$0 0000000180005ba0 f   MSVCRT:utility.obj
 0002:00000218       ?TAGGED_STATIC_INT_VALUE$initializer$@@3P6AXXZEA 0000000180006218     libHeapFilter.obj
 0002:00000220       ?TAGGED_INT_VALUE$initializer$@@3P6AXXZEA 0000000180006220     libHeapFilter.obj
 0002:00000228       ?UNTAGGED_STATIC_INT_VALUE$initializer$@@3P6AXXZEA 0000000180006228     libHeapFilter.obj
 0002:00000230       ?UNTAGGED_INT_VALUE$initializer$@@3P6AXXZEA 0000000180006230     libHeapFilter.obj
 0002:00000248       ?__scrt_initialize_tss_var@@3P6AHXZEA 0000000180006248     MSVCRT:thread_safe_statics.obj
 0002:00000370       ?opcLengths@@3QBEB         0000000180006370     libHeapFilter.obj
 0002:00002730       GS_ExceptionPointers       0000000180008730     MSVCRT:gs_report.obj
 0002:00002e58       $unwind$fprintf            0000000180008e58     libHeapFilter.obj
 0002:00002e64       $unwind$printf             0000000180008e64     libHeapFilter.obj
 0002:00002e70       $unwind$?NewObject@JNIEnv_@@QEAAPEAV_jobject@@PEAV_jclass@@PEAU_jmethodID@@ZZ 0000000180008e70     libHeapFilter.obj
 0002:00002e70       $unwind$nsk_lcomplain      0000000180008e70     libHeapFilter.obj
 0002:00002e70       $unwind$nsk_ldisplay       0000000180008e70     libHeapFilter.obj
 0002:00002e78       $unwind$nsk_jvmti_waitForSync 0000000180008e78     libHeapFilter.obj
 0002:00002e78       $unwind$nsk_lvdisplay      0000000180008e78     libHeapFilter.obj
 0002:00002e78       $unwind$set_expected_value 0000000180008e78     libHeapFilter.obj
 0002:00002e78       $unwind$_RTC_Initialize    0000000180008e78     MSVCRT:initsect.obj
 0002:00002e78       $unwind$_RTC_Terminate     0000000180008e78     MSVCRT:initsect.obj
 0002:00002e78       $unwind$?__scrt_initialize_thread_safe_statics@@YAHXZ 0000000180008e78     MSVCRT:thread_safe_statics.obj
 0002:00002e84       $unwind$nsk_complain       0000000180008e84     libHeapFilter.obj
 0002:00002e84       $unwind$nsk_printf         0000000180008e84     libHeapFilter.obj
 0002:00002e8c       $unwind$nsk_lvcomplain     0000000180008e8c     libHeapFilter.obj
 0002:00002ea4       $unwind$nsk_ltrace         0000000180008ea4     libHeapFilter.obj
 0002:00002ea4       $unwind$__report_gsfailure 0000000180008ea4     MSVCRT:gs_report.obj
 0002:00002eac       $unwind$is_primitive_type  0000000180008eac     libHeapFilter.obj
 0002:00002eac       $unwind$nsk_lvtrace        0000000180008eac     libHeapFilter.obj
 0002:00002eac       $unwind$__raise_securityfailure 0000000180008eac     MSVCRT:gs_report.obj
 0002:00002eac       $unwind$__scrt_initialize_crt 0000000180008eac     MSVCRT:utility.obj
 0002:00002eac       $unwind$__scrt_initialize_onexit_tables 0000000180008eac     MSVCRT:utility.obj
 0002:00002eac       $unwind$__scrt_release_startup_lock 0000000180008eac     MSVCRT:utility.obj
 0002:00002eac       $unwind$__scrt_uninitialize_crt 0000000180008eac     MSVCRT:utility.obj
 0002:00002eac       $unwind$_onexit            0000000180008eac     MSVCRT:utility.obj
 0002:00002eb4       $unwind$nsk_lverify        0000000180008eb4     libHeapFilter.obj
 0002:00002ec4       $unwind$nsk_vprintf        0000000180008ec4     libHeapFilter.obj
 0002:00002ed4       $unwind$?nsk_jni_lverify@@YAHHPEAUJNIEnv_@@HQEBDH1ZZ 0000000180008ed4     libHeapFilter.obj
 0002:00002ee8       $unwind$?nsk_jni_check_exception@@YAHPEAUJNIEnv_@@QEBDH@Z 0000000180008ee8     libHeapFilter.obj
 0002:00002f04       $unwind$nsk_jvmti_parseOptions 0000000180008f04     libHeapFilter.obj
 0002:00002f20       $unwind$nsk_jvmti_createJVMTIEnv 0000000180008f20     libHeapFilter.obj
 0002:00002f34       $unwind$Java_nsk_jvmti_unit_FollowReferences_FollowRefObjects_resetTags 0000000180008f34     libHeapFilter.obj
 0002:00002f34       $unwind$addRefToVerify     0000000180008f34     libHeapFilter.obj
 0002:00002f34       $unwind$nsk_jvmti_resetAgentData 0000000180008f34     libHeapFilter.obj
 0002:00002f34       $unwind$nsk_jvmti_resumeSync 0000000180008f34     libHeapFilter.obj
 0002:00002f34       $unwind$nsk_jvmti_setFailStatus 0000000180008f34     libHeapFilter.obj
 0002:00002f34       $unwind$__scrt_initialize_default_local_stdio_options 0000000180008f34     MSVCRT:default_local_stdio_options.obj
 0002:00002f34       $unwind$?dllmain_crt_dispatch@@YAHQEAUHINSTANCE__@@KQEAX@Z 0000000180008f34     MSVCRT:dll_dllmain.obj
 0002:00002f34       $unwind$DllMain            0000000180008f34     MSVCRT:dll_dllmain_stub.obj
 0002:00002f34       $unwind$__GSHandlerCheck   0000000180008f34     MSVCRT:gshandler.obj
 0002:00002f34       $unwind$?__scrt_uninitialize_thread_safe_statics@@YAXXZ 0000000180008f34     MSVCRT:thread_safe_statics.obj
 0002:00002f34       $unwind$__scrt_acquire_startup_lock 0000000180008f34     MSVCRT:utility.obj
 0002:00002f34       $unwind$__scrt_dllmain_after_initialize_c 0000000180008f34     MSVCRT:utility.obj
 0002:00002f34       $unwind$__scrt_dllmain_before_initialize_c 0000000180008f34     MSVCRT:utility.obj
 0002:00002f34       $unwind$__scrt_dllmain_crt_thread_attach 0000000180008f34     MSVCRT:utility.obj
 0002:00002f34       $unwind$__scrt_dllmain_crt_thread_detach 0000000180008f34     MSVCRT:utility.obj
 0002:00002f34       $unwind$__scrt_dllmain_uninitialize_c 0000000180008f34     MSVCRT:utility.obj
 0002:00002f34       $unwind$__scrt_dllmain_uninitialize_critical 0000000180008f34     MSVCRT:utility.obj
 0002:00002f34       $unwind$atexit             0000000180008f34     MSVCRT:utility.obj
 0002:00002f3c       $unwind$nsk_jvmti_enableEvents 0000000180008f3c     libHeapFilter.obj
 0002:00002f54       $unwind$check_option       0000000180008f54     libHeapFilter.obj
 0002:00002f54       $unwind$nsk_jvmti_findOptionValue 0000000180008f54     libHeapFilter.obj
 0002:00002f54       $unwind$_DllMainCRTStartup 0000000180008f54     MSVCRT:dll_dllmain.obj
 0002:00002f64       $unwind$nsk_jvmti_lverify  0000000180008f64     libHeapFilter.obj
 0002:00002f78       $unwind$exitOnError        0000000180008f78     libHeapFilter.obj
 0002:00002f88       $unwind$Java_nsk_share_jvmti_ArgumentHandler_getAgentOptionsString 0000000180008f88     libHeapFilter.obj
 0002:00002f9c       $unwind$Java_nsk_jvmti_unit_FollowReferences_FollowRefObjects_getTag 0000000180008f9c     libHeapFilter.obj
 0002:00002f9c       $unwind$Java_nsk_share_jvmti_DebugeeClass_checkStatus 0000000180008f9c     libHeapFilter.obj
 0002:00002f9c       $unwind$agentThreadWrapper 0000000180008f9c     libHeapFilter.obj
 0002:00002f9c       $unwind$field_callback     0000000180008f9c     libHeapFilter.obj
 0002:00002f9c       $unwind$heap_callback      0000000180008f9c     libHeapFilter.obj
 0002:00002fac       $unwind$startAgentThreadWrapper 0000000180008fac     libHeapFilter.obj
 0002:00002fc8       $unwind$syncDebuggeeStatus 0000000180008fc8     libHeapFilter.obj
 0002:00002fc8       $unwind$__scrt_dllmain_exception_filter 0000000180008fc8     MSVCRT:utility.obj
 0002:00002fdc       $unwind$Java_nsk_share_jvmti_DebugeeClass_resetAgentData 0000000180008fdc     libHeapFilter.obj
 0002:00002fe4       $unwind$MA_checkStatus     0000000180008fe4     libHeapFilter.obj
 0002:00002ff8       $unwind$Java_nsk_jvmti_unit_FollowReferences_FollowRefObjects_setTag 0000000180008ff8     libHeapFilter.obj
 0002:00003010       $unwind$Java_nsk_jvmti_unit_FollowReferences_FollowRefObjects_addRefToVerify 0000000180009010     libHeapFilter.obj
 0002:0000302c       $unwind$Agent_Initialize   000000018000902c     libHeapFilter.obj
 0002:0000304c       $unwind$string_callback    000000018000904c     libHeapFilter.obj
 0002:00003064       $unwind$array_callback     0000000180009064     libHeapFilter.obj
 0002:0000307c       $unwind$tag_objects        000000018000907c     libHeapFilter.obj
 0002:00003094       $unwind$release_object_info 0000000180009094     libHeapFilter.obj
 0002:000030ac       $unwind$verify_objects     00000001800090ac     libHeapFilter.obj
 0002:000030b4       $unwind$agent              00000001800090b4     libHeapFilter.obj
 0002:000030d0       $unwind$capture_previous_context 00000001800090d0     MSVCRT:gs_report.obj
 0002:000030dc       $unwind$__GSHandlerCheckCommon 00000001800090dc     MSVCRT:gshandler.obj
 0002:000030e8       $xdatasym                  00000001800090e8     MSVCRT:amdsecgs.obj
 0002:000030ec       $unwind$?dllmain_crt_process_attach@@YAHQEAUHINSTANCE__@@QEAX@Z 00000001800090ec     MSVCRT:dll_dllmain.obj
 0002:00003128       $unwind$?fin$0@?0??dllmain_crt_process_attach@@YAHQEAUHINSTANCE__@@QEAX@Z@4HA 0000000180009128     MSVCRT:dll_dllmain.obj
 0002:00003128       $unwind$?fin$0@?0??dllmain_crt_process_detach@@YAH_N@Z@4HA 0000000180009128     MSVCRT:dll_dllmain.obj
 0002:00003128       $unwind$?fin$1@?0??dllmain_crt_process_detach@@YAH_N@Z@4HA 0000000180009128     MSVCRT:dll_dllmain.obj
 0002:00003130       $unwind$?dllmain_crt_process_detach@@YAH_N@Z 0000000180009130     MSVCRT:dll_dllmain.obj
 0002:00003184       $unwind$?dllmain_dispatch@@YAHQEAUHINSTANCE__@@KQEAX@Z 0000000180009184     MSVCRT:dll_dllmain.obj
 0002:000031ac       $unwind$?filt$0@?0??dllmain_dispatch@@YAHQEAUHINSTANCE__@@KQEAX@Z@4HA 00000001800091ac     MSVCRT:dll_dllmain.obj
 0002:000031b4       $unwind$__scrt_is_nonwritable_in_current_image 00000001800091b4     MSVCRT:utility.obj
 0002:000031d4       $unwind$__scrt_is_nonwritable_in_current_image$filt$0 00000001800091d4     MSVCRT:utility.obj
 0002:000031dc       $unwind$__scrt_fastfail    00000001800091dc     MSVCRT:utility_desktop.obj
 0002:000031ec       $unwind$__security_init_cookie 00000001800091ec     MSVCRT:gs_support.obj
 0002:000031f8       $unwind$__isa_available_init 00000001800091f8     MSVCRT:cpu_disp.obj
 0002:00003208       $xdatasym                  0000000180009208     MSVCRT:guard_dispatch.obj
 0002:00003210       $xdatasym                  0000000180009210     MSVCRT:guard_xfg_dispatch.obj
 0002:00003220       .edata                     0000000180009220     HeapFilter.exp
 0002:00003248       rgpv                       0000000180009248     HeapFilter.exp
 0002:00003284       rgszName                   0000000180009284     HeapFilter.exp
 0002:000032c0       rgwOrd                     00000001800092c0     HeapFilter.exp
 0002:000032de       szName                     00000001800092de     HeapFilter.exp
 0002:000032ed       $N00001                    00000001800092ed     HeapFilter.exp
 0002:000032fc       $N00002                    00000001800092fc     HeapFilter.exp
 0002:00003309       $N00003                    0000000180009309     HeapFilter.exp
 0002:0000334e       $N00004                    000000018000934e     HeapFilter.exp
 0002:0000338b       $N00005                    000000018000938b     HeapFilter.exp
 0002:000033d3       $N00006                    00000001800093d3     HeapFilter.exp
 0002:00003413       $N00007                    0000000180009413     HeapFilter.exp
 0002:00003450       $N00008                    0000000180009450     HeapFilter.exp
 0002:0000348b       $N00009                    000000018000948b     HeapFilter.exp
 0002:000034b9       $N00010                    00000001800094b9     HeapFilter.exp
 0002:000034ea       $N00011                    00000001800094ea     HeapFilter.exp
 0002:00003519       $N00012                    0000000180009519     HeapFilter.exp
 0002:00003548       $N00013                    0000000180009548     HeapFilter.exp
 0002:0000357d       $N00014                    000000018000957d     HeapFilter.exp
 0002:0000358c       $N00015                    000000018000958c     HeapFilter.exp
 0002:00003a0a       .idata$6                   0000000180009a0a     kernel32:KERNEL32.dll
 0002:00003a6e       .idata$6                   0000000180009a6e     vcruntime:VCRUNTIME140.dll
 0002:00003c14       .idata$6                   0000000180009c14     ucrt:api-ms-win-crt-heap-l1-1-0.dll
 0002:00003c34       .idata$6                   0000000180009c34     ucrt:api-ms-win-crt-runtime-l1-1-0.dll
 0002:00003c56       .idata$6                   0000000180009c56     ucrt:api-ms-win-crt-convert-l1-1-0.dll
 0002:00003c78       .idata$6                   0000000180009c78     ucrt:api-ms-win-crt-stdio-l1-1-0.dll
 0002:00003c98       .idata$6                   0000000180009c98     ucrt:api-ms-win-crt-string-l1-1-0.dll
 0003:00000000       POISON                     000000018000a000     libHeapFilter.obj
 0003:00000004       ?callBytes@@3PAEA          000000018000a004     libHeapFilter.obj
 0003:00000008       ?codeAttributeName@@3PEBDEB 000000018000a008     libHeapFilter.obj
 0003:00000010       ?lineNumberAttributeName@@3PEBDEB 000000018000a010     libHeapFilter.obj
 0003:00000018       ?localVarAttributeName@@3PEBDEB 000000018000a018     libHeapFilter.obj
 0003:00000020       ?localVarTypeAttributeName@@3PEBDEB 000000018000a020     libHeapFilter.obj
 0003:00000028       ?stackMapAttributeName@@3PEBDEB 000000018000a028     libHeapFilter.obj
 0003:00000030       ?allocBytes@@3PAEA         000000018000a030     libHeapFilter.obj
 0003:00000034       filter_type                000000018000a034     libHeapFilter.obj
 0003:00000038       expected_object_count      000000018000a038     libHeapFilter.obj
 0003:00000040       TAGGED_INT_ARRAY_VALUE     000000018000a040     libHeapFilter.obj
 0003:00000048       UNTAGGED_INT_ARRAY_VALUE   000000018000a048     libHeapFilter.obj
 0003:00000050       TAGGED_STRING_VALUE        000000018000a050     libHeapFilter.obj
 0003:00000058       UNTAGGED_STRING_VALUE      000000018000a058     libHeapFilter.obj
 0003:0001ab04       UNTAGGED_INT_VALUE         0000000180024b04     libHeapFilter.obj
 0003:0001ab08       TAGGED_INT_VALUE           0000000180024b08     libHeapFilter.obj
 0003:0001ab0c       TAGGED_STATIC_INT_VALUE    0000000180024b0c     libHeapFilter.obj
 0003:0001ab10       UNTAGGED_STATIC_INT_VALUE  0000000180024b10     libHeapFilter.obj
 0003:0001ab14       redefineAttempted          0000000180024b14     libHeapFilter.obj
 0003:0001ab18       nsk_context                0000000180024b18     libHeapFilter.obj
 0003:0001ab24       redefineSucceed            0000000180024b24     libHeapFilter.obj
 0003:0001ab28       agentFailed                0000000180024b28     libHeapFilter.obj
 0003:0001ab2c       currentAgentStatus         0000000180024b2c     libHeapFilter.obj
 0003:0001ab30       context                    0000000180024b30     libHeapFilter.obj
 0003:0001abe8       agentThread                0000000180024be8     libHeapFilter.obj
 0003:0001abf0       agentThreadProc            0000000180024bf0     libHeapFilter.obj
 0003:0001abf8       agentThreadArg             0000000180024bf8     libHeapFilter.obj
 0003:0001ac00       agent_data                 0000000180024c00     libHeapFilter.obj
 0003:0001ac10       jvmti_env                  0000000180024c10     libHeapFilter.obj
 0003:0001ac18       jvm                        0000000180024c18     libHeapFilter.obj
 0003:0001ac20       jni_env                    0000000180024c20     libHeapFilter.obj
 0003:0001ac28       checkStatus_func           0000000180024c28     libHeapFilter.obj
 0003:0001ac30       ?codeAttributeIndex@@3GA   0000000180024c30     libHeapFilter.obj
 0003:0001ac34       ?lineNumberAttributeIndex@@3GA 0000000180024c34     libHeapFilter.obj
 0003:0001ac38       ?localVarAttributeIndex@@3GA 0000000180024c38     libHeapFilter.obj
 0003:0001ac3c       ?localVarTypeAttributeIndex@@3GA 0000000180024c3c     libHeapFilter.obj
 0003:0001ac40       ?stackMapAttributeIndex@@3GA 0000000180024c40     libHeapFilter.obj
 0003:0001ac44       ?stackFrameOffset@@3GA     0000000180024c44     libHeapFilter.obj
 0003:0001ac48       ?mode@@3HA                 0000000180024c48     libHeapFilter.obj
 0003:0001ac4c       ?constantPoolSize@@3GA     0000000180024c4c     libHeapFilter.obj
 0003:0001ac50       ?orig@@3PEBEEB             0000000180024c50     libHeapFilter.obj
 0003:0001ac58       ?gen@@3PEAEEA              0000000180024c58     libHeapFilter.obj
 0003:0001ac60       ?inputPos@@3PEAEEA         0000000180024c60     libHeapFilter.obj
 0003:0001ac68       ?endPos@@3PEBEEB           0000000180024c68     libHeapFilter.obj
 0003:0001ac70       ?genPos@@3PEAEEA           0000000180024c70     libHeapFilter.obj
 0003:0001ac78       ?markPos@@3PEAEEA          0000000180024c78     libHeapFilter.obj
 0003:0001ac80       ?constantPool@@3PEAPEADEA  0000000180024c80     libHeapFilter.obj
 0003:0001ac88       ?constantPoolCount@@3GA    0000000180024c88     libHeapFilter.obj
 0003:0001ac8c       ?zeroBytes@@3PAEA          0000000180024c8c     libHeapFilter.obj
 0003:0001ac90       ?codeLength@@3IA           0000000180024c90     libHeapFilter.obj
 0003:0001ac94       timeout                    0000000180024c94     libHeapFilter.obj
 0003:0001ac98       ?map@@3PEAIEA              0000000180024c98     libHeapFilter.obj
 0003:0001aca0       ?widening@@3PEACEA         0000000180024ca0     libHeapFilter.obj
 0003:0001aca8       reported_objects           0000000180024ca8     libHeapFilter.obj
 0003:0001acb0       objects_info               0000000180024cb0     libHeapFilter.obj
 0003:0001ad00       GS_ExceptionRecord         0000000180024d00     MSVCRT:gs_report.obj
 0003:0001ada0       GS_ContextRecord           0000000180024da0     MSVCRT:gs_report.obj
 0003:0001b270       ?g_tss_cv@@3U_RTL_CONDITION_VARIABLE@@A 0000000180025270     MSVCRT:thread_safe_statics.obj
 0003:0001b278       ?g_tss_event@@3PEAXEA      0000000180025278     MSVCRT:thread_safe_statics.obj
 0003:0001b280       ?g_tss_mutex@@3U_RTL_CRITICAL_SECTION@@A 0000000180025280     MSVCRT:thread_safe_statics.obj
 0003:0001b2a8       ?g_sleep_condition_variable_cs@@3P6AHPEAU_RTL_CONDITION_VARIABLE@@PEAU_RTL_CRITICAL_SECTION@@K@ZEA 00000001800252a8     MSVCRT:thread_safe_statics.obj
 0003:0001b2b0       ?g_wake_all_condition_variable@@3P6AXPEAU_RTL_CONDITION_VARIABLE@@@ZEA 00000001800252b0     MSVCRT:thread_safe_statics.obj
 0003:0001b2bc       ?__proc_attached@@3HA      00000001800252bc     MSVCRT:dll_dllmain.obj
 0003:0001b2d0       ?is_initialized_as_dll@@3_NA 00000001800252d0     MSVCRT:utility.obj
 0003:0001b2d1       ?module_local_atexit_table_initialized@@3_NA 00000001800252d1     MSVCRT:utility.obj
 0003:0001b2d8       ?module_local_atexit_table@@3U_onexit_table_t@@A 00000001800252d8     MSVCRT:utility.obj
 0003:0001b2f0       ?module_local_at_quick_exit_table@@3U_onexit_table_t@@A 00000001800252f0     MSVCRT:utility.obj
